:020000020000FC
:100000000C94574B189518951895189518951895A0
:100010001895189518951895189518951895189578
:100020001895189518951895189518951895189568
:100030001895189518951895189518950C94E32E01
:1000400018951895189518950C94E94618951895D3
:100050001895189518951895189518951895189538
:100060001895189518951895189518951895189528
:1000700018951895189518950C94C34618951895C9
:100080001895189518951895189518950D0A20002B
:100090000D0A0A205B434D2D352056657273696F3A
:1000A0006E20312E31305D000D0A20546F737320A5
:1000B0004D6F64650D0A000D0A202D3E5B44796E7C
:1000C000616D6978656C5D3A000D0A203C2D5B44DA
:1000D000796E616D6978656C5D3A000D0A203C2D82
:1000E0003E50433A00203C2D3E44796E616D697864
:1000F000656C3A000D0A2041726520796F75207396
:10010000757265203F28792F4E29000D0A205573FE
:10011000616765203A20476F205B506F736974698F
:100120006F6E20416E676C6528307830307E307895
:10013000336666295D000D0A20416C6C2044796E9F
:10014000616D6978656C27732049442077696C6C10
:100150002062652073657420746F20002E20417228
:100160006520796F7520737572653F28592F4E2968
:10017000000D0A204572726F72315B436865636BD4
:100180002044796E616D6978656C2056657273697B
:100190006F6E206973206D6F7265207468616E20C8
:1001A000335D000D0A2042284265666F7265292C76
:1001B0004E284E657874292C512851756974290090
:1001C0000D0A203438354D6F6E69746F72205B4CA8
:1001D000462C43522061726520616464656420612D
:1001E000742070617573652074696D655D0D0A001A
:1001F0000D0A204E6F20446174615B61742042726D
:100200006F61646361737420494420307846455DB2
:10021000000D0A204E6F20446174612843686563B5
:100220006B2049442C204F7065726174696E6720A1
:100230004D6F64652C20426175642072617465297C
:1002400000204C454E3A000D0A204C454420426C9B
:10025000696E6B2049443A002044796E616D69787B
:10026000656C7320466F756E642E000D0A204C4538
:100270004420426C696E6B2049443A000D20466F61
:10028000756E642120424155445F5245473A002C27
:100290002049443A000D0A20426175642052656786
:1002A000206973206368616E67656420746F200045
:1002B000425053000D0A2049443A30202D20000DB1
:1002C0000A2044656C61793A000D0A20546F7271FE
:1002D000756520456E61626C65000D0A204D6F7674
:1002E000652030203C2D3E203078336666000D0AB4
:1002F00020416E79204B657920746F20436F6E74B6
:10030000696E75652E2E2E000D0A205B45455052F4
:100310004F4D20415245415D0D0A204D4F44454C03
:100320005F4E554D4245525F4C202020202020201A
:1003300020285229205B000D0A204D4F44454C5F78
:100340004E554D4245525F4820202020202020203D
:10035000285229205B000D0A2056455253494F4E22
:100360002020202020202020202020202020202885
:100370005229205B000D0A20494420202020202003
:100380002020202020202020202020202028522F24
:1003900057295B000D0A20424155445F52415445A4
:1003A00020202020202020202020202028522F57CD
:1003B000295B000D0A2052455455524E5F44454C6E
:1003C00041595F54494D452020202028522F57295C
:1003D0005B000D0A2043575F414E474C455F4C4937
:1003E0004D49545F4C202020202028522F57295B54
:1003F000000D0A2043575F414E474C455F4C494D25
:1004000049545F48202020202028522F57295B0084
:100410000D0A204343575F414E474C455F4C494DC1
:1004200049545F4C2020202028522F57295B000D73
:100430000A204343575F414E474C455F4C494D4965
:10044000545F482020202028522F57295B000D0A96
:10045000202852455345525645442920202020202B
:1004600020202020202028522F57295B000D0A2011
:100470004C494D49545F54454D5045524154555295
:10048000452020202028522F57295B000D0A2044A8
:100490004F574E5F4C494D49545F564F4C5441475E
:1004A0004520202028522F57295B000D0A20555047
:1004B0005F4C494D49545F564F4C544147452020AD
:1004C00020202028522F57295B000D0A204D41582B
:1004D0005F544F525155455F4C2020202020202052
:1004E000202028522F57295B000D0A204D41585FCC
:1004F000544F525155455F48202020202020202075
:100500002028522F57295B000D0A2052455455527E
:100510004E5F4C4556454C20202020202020202096
:1005200028522F57295B000D0A20414C41524D5F44
:100530004C4544202020202020202020202020283E
:10054000522F57295B000D0A20414C41524D5F53F9
:10055000485554444F574E20202020202020285218
:100560002F57295B000D0A20285245534552564506
:100570004429202020202020202020202028522F05
:1005800057295B000D0A20444F574E5F43414C49A9
:1005900042524154494F4E5F4C20202028522F5741
:1005A000295B000D0A20444F574E5F43414C49429E
:1005B000524154494F4E5F4820202028522F57293E
:1005C0005B000D0A2055505F43414C494252415453
:1005D000494F4E5F4C202020202028522F57295B66
:1005E000000D0A2055505F43414C49425241544945
:1005F0004F4E5F48202020202028522F57295B0093
:100600000D0A205B52414D20415245415D0D0A20AB
:10061000544F525155455F454E41424C4520202094
:10062000202020202028522F57295B000D0A204C23
:100630004544202020202020202020202020202071
:100640002020202028522F57295B000D0A204357D5
:100650005F434F4D504C49414E43455F4D415247DA
:10066000494E2028522F57295B000D0A204343573B
:100670005F434F4D504C49414E43455F4D415247BA
:10068000494E28522F57295B000D0A2043575F43DC
:100690004F4D504C49414E43455F534C4F504520C0
:1006A0002028522F57295B000D0A204343575F43F0
:1006B0004F4D504C49414E43455F534C4F504520A0
:1006C00028522F57295B000D0A20474F414C5F509D
:1006D0004F534954494F4E5F4C2020202020202862
:1006E000522F57295B000D0A20474F414C5F504F56
:1006F000534954494F4E5F48202020202020285243
:100700002F57295B000D0A204D4F56494E475F5326
:10071000504545445F4C2020202020202028522F87
:1007200057295B000D0A204D4F56494E475F5350E5
:100730004545445F482020202020202028522F5764
:10074000295B000D0A20544F525155455F4C494DCD
:1007500049545F4C2020202020202028522F572948
:100760005B000D0A20544F525155455F4C494D498D
:10077000545F482020202020202028522F57295B1A
:10078000000D0A2050524553454E545F504F534977
:1007900054494F4E5F4C20202020285229205B00D6
:1007A0000D0A2050524553454E545F504F53495403
:1007B000494F4E5F4820202020285229205B000D01
:1007C0000A2050524553454E545F53504545445FAF
:1007D0004C20202020202020285229205B000D0AB8
:1007E0002050524553454E545F53504545445F4851
:1007F00020202020202020285229205B000D0A20C4
:1008000050524553454E545F4C4F41445F4C20205D
:10081000202020202020285229205B000D0A205073
:10082000524553454E545F4C4F41445F4820202071
:100830002020202020285229205B000D0A20505221
:100840004553454E545F564F4C5441474520202058
:1008500020202020285229205B000D0A20505245DC
:1008600053454E545F54454D5045524154555245A1
:10087000202020285229205B000D0A20524547499C
:100880005354455245445F494E53545255432E20CC
:100890002028522F57295B000D0A205245534552FC
:1008A0005645442850415553455F54494D452920EC
:1008B00028522F57295B000D0A204D4F56494E47AD
:1008C0002020202020202020202020202020202028
:1008D000285229205B000D0A204C4F434B2020203A
:1008E00020202020202020202020202020202852CE
:1008F0002F57295B000D0A2050554E43485F4C206E
:100900002020202020202020202020202028522F9E
:1009100057295B000D0A2050554E43485F48202060
:1009200020202020202020202020202028522F5747
:10093000295B000D0A0A2044554D50284429203ACD
:100940002044756D7020636F6E74726F6C207461DB
:10095000626C652E000D0A204944205B49445F4EBD
:10096000554D5D203A20536574204944206F662020
:1009700064796E616D6978656C2E000D0A204349BB
:1009800044205B49445F4E554D5D203A20436861E9
:100990006E676520436F6E74726F6C2049442E0041
:1009A0000D0A2052454144205B414444525D5B4C5A
:1009B000454E5D203A205265616420646174612E69
:1009C0002065782952656164203130203220285218
:1009D0006561642066726F6D20307831302C206C38
:1009E000656E677468203229000D0A2057524954F9
:1009F00045205B414444525D5B44415441315D2E8E
:100A00002E203A20577269746520646174612E202B
:100A100065782957726974652031342C3120285744
:100A20007269746520312061742030783134290076
:100A30000D0A205245475F5752205B414444525DA6
:100A40005B44415441315D2E2E203A205265676946
:100A50007374657220777269746520696E7374753A
:100A6000726374696F6E000D0A20414354494F4E02
:100A7000203A20416374696F6E205245475F575298
:100A800020696E737472756374696F6E000D0A204D
:100A9000476F205B504F534954494F4E5D5B535055
:100AA0004545445D3A20476F746F20746865207037
:100AB0006F736974696F6E207769746820746865F4
:100AC0002073706565642E000D0A20484558205B30
:100AD0004E554D5D5B4E554D5D2E2E2E203A2054C9
:100AE00072616E736D6974652072617720646174E0
:100AF000612E2065782948657820464620464620A4
:100B00003031203033000D0A205245534554203AED
:100B10002044796E616D6978656C205265736574E7
:100B20002E000D0A2050494E47205B4E554D5D3A30
:100B3000206578292050696E67204E554D20494424
:100B40002064796E616D6978656C2E000D0A205302
:100B50005752205B414444525D5B4C454E5D5B49BE
:100B6000445D5B444154415D2E2E2E5B49445D5BE8
:100B7000444154415D2E2E2E203A2053796E63203D
:100B800057726974652E000D0A205343414E205B55
:100B90004E554D5D203A205343414E206C696E6B9B
:100BA00065642064796E616D6978656C20696E207A
:100BB000307E4E554D20696E2063757272656E747D
:100BC000206261756420726174652E000D0A204CEC
:100BD0004544205B4E554D5D203A20426C696E6B5A
:100BE000204C4544206F66204E554D2049442E2010
:100BF0002742272C274E2720666F72204944206306
:100C000068616E67652E2027512720666F7220511C
:100C10007569742E000D0A2042415544205B4E55E3
:100C20004D5D203A205365742062617564207261C5
:100C300074652020657829204241554420323228AD
:100C40003537363030425053292C2042415544200C
:100C50003128314D42505329000D0A20534541524D
:100C60004348203A205365617263682049442061FB
:100C70006E64206261756472617465206F662061C4
:100C80006C6C206C696E6B65642064796E616D6953
:100C900078656C732E000D0A2055706461746520B0
:100CA0005B53544152545F49445D205B454E445F61
:100CB00049445D203A2044796E616D6978656C2005
:100CC0006669726D77617265207570646174652EF6
:100CD0002873797374656D2075736572206F6E6CFF
:100CE0007929000D0A0A2020202020202020436F8F
:100CF0007079726967687420524F424F544953208B
:100D0000434F2E2C4C54442E0D0A005B496E7661E5
:100D10006C6964205061676520526561643A000D1A
:100D20000A205B4572723A5278442054696D656FAF
:100D300075745D000D0A205B4572723A57726F6ED2
:100D400067204865616465725D000D0A205B45722D
:100D5000723A5478494420213D20527849445D003C
:100D60000D0A205B4572723A57726F6E67204C65B0
:100D70006E6774685D000D0A205B4572723A5772A7
:100D80006F6E6720436865636B53756D5D000D0A78
:100D900020555044415445205B53544152542049FE
:100DA000445D205B454E442049445D005D3A000DA2
:100DB0000A2049443A00205374616E6462792E001F
:100DC0002057726974696E672E2E00205375636315
:100DD0006573732E00204572726F722E000D0A200B
:100DE0004572722049443A002042616420436F6D8D
:100DF0006D616E64005B457869745D000D0A204D7D
:100E00004F54494F4E20504C4159205041474520A6
:100E100020202028522F5729000D0A204F4E205005
:100E20004C4159494E47204D4F54494F4E202020A8
:100E30002028522920000D0A205458205749524595
:100E40004C455353205041434B4554202028522FAA
:100E50005729000D0A20525820574952454C4553F6
:100E600053205041434B4554202020285229200034
:100E70000D0A204E4557205041434B4554204152C6
:100E8000524956454420202028522920000D0A208E
:100E9000415558204C45442020202020202020204F
:100EA0002020202028522F5729000D0A2042555477
:100EB000544F4E282D532D552D442D4C2D52292065
:100EC000202028522920000D0A2054494D4552283F
:100ED0003132356D5365632045616368292028529E
:100EE0002F5729000D0A205A4947424545204944B9
:100EF000202020202020202020202028522F572969
:100F0000000D0A20524F424F5420494420202020F7
:100F1000202020202020202028522F5729000D4457
:100F2000796E616D6978656C2020302830783030BA
:100F3000295B202020205D000D0A44796E616D69D7
:100F400078656C2020312830783031295B202020D2
:100F5000205D0020506167654E756D6265723A00D4
:100F60000D0A44796E616D6978656C2020322830F5
:100F7000783032295B202020205D0020416464729B
:100F80003A000D0A44796E616D6978656C202033F2
:100F90002830783033295B202020205D0020285223
:100FA0006573657276656429203A000D0A44796E8E
:100FB000616D6978656C2020342830783034295B85
:100FC000202020205D00202020506C6179436F7527
:100FD0006E743A000D0A44796E616D6978656C2013
:100FE00020352830783035295B202020205D0020F6
:100FF00028526573657276656429203A000D0A44AB
:10100000796E616D6978656C2020362830783036CD
:10101000295B202020205D002028526573657276B0
:10102000656429203A000D0A44796E616D6978651E
:101030006C2020372830783037295B202020205D35
:10104000002028526573657276656429203A000D88
:101050000A44796E616D6978656C20203828307893
:101060003038295B202020205D00202852657365E0
:101070007276656429203A000D0A44796E616D69C3
:1010800078656C2020392830783039295B20202081
:10109000205D002020205061676520537465703A00
:1010A000000D0A44796E616D6978656C20313028D5
:1010B00030783041295B202020205D0020436F6E76
:1010C00074726F6C436F64653A000D0A44796E6107
:1010D0006D6978656C2031312830783042295B2089
:1010E0002020205D002020506167652053706565D9
:1010F000643A000D0A44796E616D6978656C20313F
:10110000322830783043295B202020205D002020C9
:101110002044584C2053657475703A000D0A447988
:101120006E616D6978656C203133283078304429E0
:101130005B202020205D002020416363656C2054EB
:10114000696D653A000D0A44796E616D6978656C68
:101150002031342830783045295B202020205D0064
:101160004C696E6B20746F204E6578743A000D0ADE
:1011700044796E616D6978656C203135283078303E
:1011800046295B202020205D004C696E6B20746F27
:1011900020457869743A000D0A44796E616D69786A
:1011A000656C2031362830783130295B20202020B2
:1011B0005D002852657365727665645031293A0086
:1011C0000D0A44796E616D6978656C20313728307D
:1011D000783131295B202020205D0028526573651D
:1011E000727665645231293A000D0A44796E616D58
:1011F0006978656C2031382830783132295B2020BD
:1012000020205D002852657365727665645032292E
:101210003A000D0A44796E616D6978656C20313948
:101220002830783133295B202020205D002852654A
:101230007365727665645232293A000D0A44796EFC
:10124000616D6978656C2032302830783134295BE3
:10125000202020205D000D0A44796E616D6978655B
:101260006C2032312830783135295B202020205DF8
:10127000000D0A44796E616D6978656C2032322800
:1012800030783136295B202020205D000D0A44791A
:101290006E616D6978656C2032332830783137297A
:1012A0005B202020205D000D0A44796E616D697815
:1012B000656C2032342830783138295B202020209A
:1012C0005D000D0A44796E616D6978656C20323578
:1012D0002830783139295B202020205D000D0A4418
:1012E000796E616D6978656C2032362830783161AD
:1012F000295B202020205D000D0A44796E616D6914
:1013000078656C2032372830783162295B202020C4
:10131000205D000D0A44796E616D6978656C20323C
:10132000382830783163295B202020205D000D0AA9
:1013300044796E616D6978656C2032392830783176
:1013400064295B202020205D000D0A44796E616DC8
:101350006978656C2033302830783165295B20202E
:1013600020205D000D0A20202050617573655469AE
:101370006D65202020202020205B2020205D000D96
:101380000A20202053706565642020202020202022
:10139000202020205B2020205D20202020202020D5
:1013A000202020202020202020202020202020203D
:1013B000202020202020202020202020205B583AA0
:1013C0002D2D2C593A2D2D2C413A2D2D2D2D5D00F2
:1013D0000D0A202020202020202020202020202036
:1013E00020202020205354503720205354503020A8
:1013F00053545031205354503220535450332053BF
:10140000545034205354503520535450362020200B
:1014100020476F20537465703A2020202020000D53
:101420000A202020202020202020202020202020D2
:10143000202020202020202020204D5354522053B3
:101440004C4156204F46535420202020202020205D
:10145000202020202020202020202020202020208C
:10146000476F20537465703A2020202020000D0A19
:101470005D205F20202020202020202020202020F0
:10148000202020202020202020202020202020205C
:10149000202020202020202020202020202020204C
:1014A000202020202020202020202020202020203C
:1014B00020202020202020202020202000204172D9
:1014C0006520796F7520737572653F5B792F4E5D6E
:1014D0000020496E76616C69642050616765002068
:1014E000496E76616C696420506172616D657465E6
:1014F0007200204F66667365742055706461746570
:101500006400204F7574206F662052616E6765001D
:10151000204F4B000D0A20202020202020202D438A
:101520004D3A2052503D2850617261302C4F502C62
:10153000506172613129204C4B205253205B414451
:1015400044525D2020000D0A20427265616B2061CB
:101550007420000D0A204552524F523A004946204D
:101560002020202000454C534520494600454C533F
:101570004520202000616E642F6F7220004A554D77
:1015800050202020004C4F414420202000434F4D4C
:1015900050555445005354415254202000454E4468
:1015A000202020200043414C4C2020200052455454
:1015B00055524E20004E554C4C202020000D0A2044
:1015C0004845584120444953504C4159204D4F44BF
:1015D00045000D0A20444543494D414C20444953A0
:1015E000504C4159204D4F44450003404C464D4816
:1015F00040454A230102030A222121217D7D7D7D70
:101600007D7D7D7D7D7D7D7D7D7D7D797673716E3A
:101610006C6967656361605E5C5B595857555453EC
:1016200051504F4E4D4C4B4A494847464544434222
:101630004241403F3F3E3D3C3C3B3A3939383737E9
:101640003636353434333332313130302F2F2E2D7E
:101650002D2C2C2B2B2A2A292928282727262625FA
:10166000252524242323222221212020201F1F1E60
:101670001E1D1D1D1C1C1B1B1A1A1A1919181818BF
:101680001717161616151514141413131212121117
:10169000111010100F0F0E0E0E0D0D0C0C0C0B0B6D
:1016A0000A0A0909090808070707060605050404C8
:1016B0000403030202010101000000000000000019
:1016C000000000000000000000000000000000001A
:1016D000000000000000000000000000000000000A
:1016E00000000000000000000000000000000000FA
:1016F00000000000000000000000000000000001E9
:1017000001010200020001010101020001010101C9
:1017100002000200010101010101020002000200B9
:1017200002000200020001010101010102000101A9
:10173000020002000000000101010101000001019E
:10174000010101000101010101010000010100008E
:101750000000000001000000010102000101000082
:1017600001010101020002000101682FA901812F7E
:101770000023B9F40FE003BF00E002BF09E01DE35E
:101780000E94AF4B10E0003021E0120710F000E0A3
:1017900009C001BF082F00FB07B701F907BF01E02F
:1017A00001C000E0862F089500E00093610002B9B7
:1017B00001BB04BB07BB0ABB00E0009365000093BC
:1017C000620003B902BB05BB08BB00B50B7F00BDBF
:1017D00000B50B7F00BD00E00093610002B901BBC2
:1017E00004BB07BB0ABB00E00093650000936200E6
:1017F00003B902BB05BB08BBBD9AC59A909A1C9A57
:101800001D9A1E9A1F9A04B30F6704BB02B10C60A5
:1018100002B9AC9AAB9AAA9AA99AA89AAE9AAD9A2A
:10182000AC9AAB9AAA9AA99AA89A1A981B9A01B349
:10183000006701BB9798949A959A9698AC9AAB9A40
:10184000AA9AA99AA89A0895002391F400E0009317
:10185000900019B902E00BB908E10AB920FB0EF4B7
:10186000579A06E0009395000FEF0CB95E9A089521
:101870000130E9F400E0009398001093990002E031
:1018800000939B0008E100939A0020FB2EF4009146
:101890009A00006800939A0006E000939D000FEF05
:1018A00000939C0000919B00006400939B000895AE
:1018B000592F482F80E090E008C02FE93FE02150E9
:1018C0003040E9F700C00000019680179107A8F3A7
:1018D000842F952F08959A938A9380E090E083D285
:1018E0000A3318F00753102F02C00053102F012F96
:1018F00010E0102F00E0110F110F110F110F802BAE
:10190000912B71D20A3318F00753102F02C00053E5
:10191000102F012F302F20E0822B932B64D20A331B
:1019200018F00753102F02C00053102F012F10E0A2
:1019300044E00E94A34B802B912B55D20A3318F020
:101940000753102F02C00053102F012F10E0802BDF
:10195000912B8C018991999108950E94454C229771
:1019600028833983B02FD12E7A0182E090E001E004
:101970000093DA0CBB249699B394CC249599C39424
:10198000969A959825C0949801E010E091DF00E0C8
:101990000093F00C0093EF0C949A05E010E088DFC0
:1019A00001E2F0D001E311E083DF08E0EBD0009129
:1019B000EF0C1091F00C011751F00091EF0C109109
:1019C000F00C011721F00FD20132B9F791E08A959E
:1019D000813010F09923B9F2992309F49CC000E0FA
:1019E0000093F00C0093EF0C4424552466247724D4
:1019F000A0E08824992409E6C5D008E0C3D0F3D13B
:101A00000A33E9F7F0D10A33E9F765DF2801EBD1B2
:101A10000A33E9F760DF38010FEF60160FEF700649
:101A200049F0E1D10A33E9F7DED1093511F4A1E03B
:101A300001C0A0E00EE110E03BDF00E00093F00CFD
:101A40000093EF0C02E59ED008E09CD0CCD1802F13
:101A50008C3641F4C8D10A33E9F73DDF4801AA24A6
:101A6000A39403C08F3691F7AA24E4EDFCE04082F2
:101A70005182E6EDFCE060827182E8EDFCE080825C
:101A80009182B0FBC6F404E110E012DF04E47AD0E6
:101A900008E078D0A8D10A33E9F705E010E008DFC4
:101AA0000881198176D108E06DD008E06BD008E09C
:101AB00069D008E067D0B1FB4EF404E110E0F8DE35
:101AC000DA1621F007E55ED008E05CD0B2FBCEF478
:101AD000AA20B9F004E110E0EBDE03E453D008E003
:101AE00051D081D10A33E9F705E010E0E1DE87014A
:101AF00050D108E047D008E045D008E043D008E0E6
:101B000041D004E110E0D4DE05E43CD008E03AD056
:101B100005E010E0CDDE00E00093F00C0093EF0C48
:101B20000B2D00FD969A00FF96980C2D00FD959ABE
:101B300000FF959800E00093DA0C092F2296E0E16F
:101B40000C94564C5E9A1B981A9A18D05E9BFECF46
:101B50001A981B9A08958A93802F082F02950F7068
:101B6000005D0A3308F0095F0DD08F70805D082F8B
:101B70000A3308F0095F06D0899108955D9BFECF76
:101B80000CB90895A99810919B00212F25FFFBCF38
:101B900000939C0008959A938A93802F082F44E61F
:101BA0000E94854B902F092F005DECDF04E6909F8B
:101BB0008019082F4AE00E94854B902F092F005D65
:101BC000E1DF0AE0909F8019805D082FDBDF8991BB
:101BD000999108950E94474C48015901DD24BB208A
:101BE00052F49094A094B094000B8194900AA00AAF
:101BF000B00A0DE2C7DF80E09AECAAE9BBE3CC248F
:101C00001AC0DD2019F08201005DBCDF8201930162
:101C1000AC01BD010E94D44B801A910AA20AB30AFA
:101C20008C019D014AE050E060E070E00E941E4C93
:101C3000C801D901C39409E0C016A8F48401950134
:101C4000AC01BD010E941E4C402E55246624772411
:101C5000042D052906290729A1F28201005D92DFE2
:101C6000DD24D394D3CF84019501AC01BD010E9442
:101C70001E4C402E552466247724042D005D82DFFF
:101C8000EEE00C94584C0E944D4C38015524A0E1D4
:101C9000B7E244240FC000E375DF8C01AD010E9460
:101CA000934B601A710A8D014AE050E00E94AF4BDD
:101CB000D801439405E04016D0F48301AD010E94A1
:101CC000AF4BC801082F092B31F0082F005D5ADFF8
:101CD00055245394E2CF552021F0082F005D52DFA8
:101CE000DCCF04E04016B8F600E24CDFD6CFE8E0E7
:101CF0000C945E4C10915209112311F02CDF0895C1
:101D000023E010E00AD0089520915209222311F017
:101D100040D0089524E001D008950E944B4C380132
:101D2000822E5524A0E1B7E244240FC000E32ADF4D
:101D30008C01AD010E94934B601A710A8D014AE03B
:101D400050E00E94AF4BD801439405E04016F0F4F8
:101D50008301AD010E94AF4BC80104E010E0242DC7
:101D600030E0021B130B9924081519050CF7082FF6
:101D7000092B31F0082F005D05DF55245394D8CF8F
:101D80005520A1F2082F005DFDDED2CFEAE00C94D1
:101D90005C4C9A938A93C8018C01012F10E0DBDE22
:101DA000082FD9DE8991999108950E94514CC8015C
:101DB000D9018C019D01022F132F330F220B330BFE
:101DC000E8DF8C01E6DFE4E00C94624CBA93AA935E
:101DD000D80103C00C91D6DE11960C910023D1F7E7
:101DE000A991B99108950091F00C1091EF0C011791
:101DF000D1F30091F00C102F13951093F00C10E01C
:101E00000F701070F801EF50F34F008108958A931E
:101E1000802F082FC0DE08E2B5DE00E3B3DE08E560
:101E2000B1DE082F98DE09E2ADDE899108950E94A7
:101E30004A4CEF97EF97EF972797A898992401E0DE
:101E400000935B0901E000935A0905C004E110E02A
:101E50002FDD08E001BD992011F00C9480170EE9E8
:101E600015E0B4DF00914B09D2DF07EA15E0AEDFE1
:101E700020E08E0108571F4F0E94311F00E00883A9
:101E8000AE0148575F4F9E01205F3F4F8E010E9479
:101E9000851D802E00915809009359098820D9F298
:101EA0000FE1801610F00EE1802E28E436E08E015E
:101EB0000E94631D002351F626E436E08E010E9445
:101EC000631D002309F450C007EB10E00E94904905
:101ED00080E01CC0FE017096082F10E0000F111F5B
:101EE000000F111FE00FF11F00811181228133814A
:101EF00090E0FC01E254F74F008390E0FC01E254D3
:101F0000F74F0081F7DE00E23DDE839590E0E82D9B
:101F1000F0E031978E179F07ECF21B981A9A80E039
:101F200008C090E0FC01E254F74F008127DE5E9A82
:101F3000839590E0E82DF0E031978E179F078CF3A2
:101F40005E9BFECF1A981B9A0FEF0E943C470093AE
:101F50005C0909EC10E00E94904920915C090AE0BC
:101F600018E00E94494877CF21E436E08E010E94B4
:101F7000631D002371F42EE336E08E010E94631D81
:101F8000002339F42CE935E08E010E94631D002303
:101F900069F100914B09083CB1F40CE810E00E9493
:101FA0009049088919892A893B8931DF0AE3EADDEA
:101FB000088919892A893B89102F00914B090E94B1
:101FC0009C3AA2DE48CF088919892A893B89009367
:101FD00088070C891D892E893F890093890722E093
:101FE00012E000914B090E94734835CF27E935E094
:101FF0008E010E94631D0023A9F014E300914B0998
:102000000E942C4BC801282F14E100914B090E941B
:10201000FD1C892F90E0282F15E100914B090E94AB
:10202000FD1C19CF23E935E08E010E94631D0023BA
:1020300041F001E0009352090DEB15E10E94904937
:102040000ACF2FE835E08E010E94631D002341F086
:1020500000E00093520902ED15E10E949049FBCE89
:102060002AE835E08E010E94631D0023A9F014E3E5
:1020700000914B090E942C4BC801282F16E10091BA
:102080004B090E94FD1C892F90E0282F17E1009139
:102090004B090E94FD1CDFCE26E835E08E010E9430
:1020A000631D002339F42EE735E08E010E94631D85
:1020B0000023F9F080E014C0FE017096082F10E0B4
:1020C000000F111F000F111FE00FF11F0081118180
:1020D0002281338190E0FC01E857F84F008383951B
:1020E000881550F38A94282D13E80EEF0E94734848
:1020F000B2CE28E735E08E010E94631D002371F403
:1021000025E735E08E010E94631D002339F423E7A3
:1021100035E08E010E94631D0023A1F100914B095F
:10212000083C81F40C891D892E893F8998014889D2
:1021300059896A897B898A01102F00914B090E9475
:10214000903989CE80E014C0FE017096082F10E00F
:10215000000F111F000F111FE00FF11F00811181EF
:102160002281338190E0FC01E857F84F008383958A
:10217000881550F38A94282D13E000914B090E9492
:10218000734869CE2CE635E08E010E94631D002362
:1021900001F180E014C0FE017096082F10E0000FDE
:1021A000111F000F111FE00FF11F0081118122810B
:1021B000338190E0FC01E857F84F00838395881540
:1021C00050F38A94282D14E000914B090E94734823
:1021D00042CE25E635E08E010E94631D002339F4CE
:1021E00021E635E08E010E94631D0023F9F080E0B6
:1021F00014C0FE017096082F10E0000F111F000F91
:10220000111FE00FF11F008111812281338190E0C5
:10221000FC01E857F84F00838395881550F38A94A2
:10222000282D15E00EEF0E94734815CE2AE535E003
:102230008E010E94631D002381F00C891D892E8967
:102240003F89202F488959896A897B898A01102F03
:1022500000914B090E94FD1CFECD24E535E08E0166
:102260000E94631D002321F104EF10E00E949049B9
:10227000BADD093719F0093509F0EDCD01E0801616
:1022800019F400914B0904C0088919892A893B89EE
:1022900020E016E00E947348002309F4DCCD01E041
:1022A00000934B0921E030E0A9010E94814BD3CD7E
:1022B0002DE435E08E010E94631D0023A1F001E0B2
:1022C000801639F420E017E000914B090E94734812
:1022D000C2CD20E017E0488959896A897B89042F9B
:1022E0000E947348B8CD2AE435E08E010E94631D38
:1022F000002339F428E435E08E010E94631D002399
:10230000D9F102E0801619F003E0801681F50EE1A4
:1023100000938807088919892A893B8900938907CE
:10232000088919892A893B89012F10E000938A07BF
:1023300003E08016A9F40C891D892E893F8900933A
:102340008B070C891D892E893F89012F10E000938E
:102350008C0725E013E000914B090E9473487BCD68
:1023600023E013E000914B090E94734874CD0BE009
:1023700011E00E9490496FCD23E435E08E010E9468
:10238000631D002379F001E0801619F400914B09D8
:1023900004C0088919892A893B8920E011E00E943C
:1023A000734859CD20E435E08E010E94631D00235F
:1023B00049F103E000938807088919892A893B8934
:1023C0000093890706E311E00E9490490091890774
:1023D00091DC0CE511E00E94904905DD093519F00A
:1023E000093709F038CD22E013E00EEF0E94734860
:1023F0000091890700934B0921E030E0A9010E9478
:10240000814B29CD2DEF35E08E010E94631D002305
:1024100039F42BEF35E08E010E94631D0023E1F0BB
:1024200000914B09083C11F4BED515CD00E0009396
:1024300088070AE30093890722E012E000914B0924
:102440000E947348002309F406CD00914B090E3F0A
:1024500009F401CDA8D5FFCC24EF35E08E010E9410
:10246000631D002309F43FC103E0801651F448883E
:1024700059886A887B880C891D892E893F89A02EFE
:102480000DC002E0801631F4488859886A887B883C
:10249000A42C04C00EE81DE00E94904902E08016C2
:1024A00021F003E0801609F0D6CC00E000935A0931
:1024B00000935B0909B1023289F421E014E00EEFC8
:1024C0000E94424B0AE010E0F3D901E009B9009301
:1024D0004A0920E030E0A9010E94814B22E214E089
:1024E0000EEF0E94424B0AE010E0E2D902E209B985
:1024F00000934A0920E030E0A9010E94814B00E0EE
:102500000E94AB4905C001E711E00E949049439445
:10251000A41408F4DAC05524F201E35AF64F0081FE
:102520000023A9F30FEA1DE00E949049042DE2DB8D
:1025300090E0992399F491E080E08F31D0F7082F53
:102540000E94351D002341F020E011E0082F0E9479
:102550007348002309F490E08395EFCF06EB1DE06C
:102560000E94904980E00FC0841561F090E0FC016A
:10257000E35AF64F0081002329F025E01DE2082FE1
:102580000E94FD1C83958F3178F300EC1DE00E94C2
:1025900090492FEF1AEF042D0E94FD1C2EEF1DE233
:1025A000042D0E94FD1C002309F4ADCF04E610E0C9
:1025B0007FD90DE0C7DA00E00E94B71C0CE4C2DA54
:1025C00000E00E94B71C1B981A9A80E090ECA0E0F3
:1025D000B0E055246624772412C0FC013A2F3BBF9B
:1025E000069000E00BBF8F5F9F4FAF4FBF4F500C67
:1025F000002DC4DA5E9A01E0600E00E0701E0FEF5D
:10260000601607E1700648F3052DB8DA5E9A5E9B06
:10261000FECF1A981B9A00E00E94B71C06E592DADA
:1026200000E00E94B71C00E001C00395043638F4B6
:1026300010E0F801E65FF74F10811D32B1F7039506
:10264000202F01C00395043638F410E0F801E65F4E
:10265000F74F10811D32B1F7039510E001C01395BB
:10266000183090F4602F062F0395422F242F2395C6
:1026700070E0FB01E65FF74F308150E0FA01E65F62
:10268000F74F4081341759F31830D1F40BEC1DE0AB
:102690000E94904901E456DA00E00E94B71C07E46A
:1026A00051DA00E00E94B71C20E017E0042D0E94E0
:1026B00073480CE211E0FCD800E000935A0927CFE0
:1026C00005ED1DE00E94904922CF0E94594909B1B1
:1026D00000934A0920E030E0A9010E94814B01E00B
:1026E00000935B09B8CB2FEE35E08E010E94631D8D
:1026F000002309F440C0B0915A0900E000935B093F
:1027000000935A0980E001E0801611F4AEEF05C095
:10271000088919892A893B89A02F0CE810E00E94BA
:10272000904990E005C00DE22DDA0DE52BDA939586
:102730009A1788F40BE526DA092FDCDA0AE322DAA5
:1027400020E011E0092F0E947348002361F30FE499
:1027500019DA8395EACF0CE810E00E949049082F1F
:1027600056DB08E512E00E949049B0935A0901E057
:1027700000935B0970CB2BEE35E08E010E94631D48
:10278000002309F459C001E0801619F4A0914B0907
:1027900005C0088919892A893B89A02F00E0009388
:1027A0005B0900935A0903EA11E00E94904980E016
:1027B00007E412E00E9490490A2F9CDA0091F00C85
:1027C0001091EF0C011791F00EDB802F823411F085
:1027D000823609F4AA958E3411F08E3609F4A39549
:1027E0000BE612E00E9490490A2F84DA09E1009377
:1027F000880701E00093890722E013E00A2F0E9476
:10280000734804E610E054D809E10093880700E01B
:102810000093890722E013E00A2F0E94734804E620
:1028200010E046D8813521F0813711F08B3131F637
:1028300001E000935B090FCB24EE35E08E010E948E
:10284000631D002309F48EC000E000935B090AE0D9
:1028500099D980E001C083958E3F08F078C089B98E
:1028600020E011E00EEF0E9473480DE08BD980FB51
:102870001EF40BE287D902C00AE284D900915C09F8
:10288000002309F45DC0A0E056C0B0E0FD01E65FA2
:10289000F74F00810F3F09F04DC00A2F10E00F5F86
:1028A0001F4FF801E65FF74F00810F3F09F042C06C
:1028B0000A2F10E00D5F1F4FF801E65FF74F008110
:1028C0000230C1F50A2F10E00E5F1F4FF801E65FDE
:1028D000F74F408150E00A2F10E00D5F1F4FF801C5
:1028E000E65FF74F208130E0240F351F0A2F10E0FC
:1028F0000B5F1F4FF801E65FF74F008110E0020FFA
:10290000131F0F3F20E01207A9F40CE712E00E940A
:102910009049082FEFD90FE812E00E9490490A2F42
:1029200010E00E5F1F4FF801E65FF74F0081E2D91C
:102930000AE028D9A39500915C09A01708F4A5CF57
:102940000091F00C1091EF0C011709F484CF009165
:102950004A0909B901E000935B090DE013D900E2CF
:1029600011D979CA2FED35E08E010E94631D002335
:1029700091F104E000938807088919892A893B8925
:102980000093890722E013E00EEF0E94734805E9E7
:1029900012E00E94904900E814E82EE130E04889F6
:1029A00059896A897B894F5F5F4F6F4F7F4F0E94C4
:1029B000F84B10D900EB12E00E9490490889198960
:1029C0002A893B8909B900934A0920E030E0A9012E
:1029D0000E94814B40CA27ED35E08E010E94631DA5
:1029E000002309F442C001E0801631F400E1402EDA
:1029F00055246624772404C0488859886A887B88CF
:102A000000EC11E00E9490492BC0009159091091EF
:102A100058090117A1F080E090E0A0E0B0E0AA24FE
:102A20000091590910E0F801E857F94F0081E9E5F4
:102A3000F9E01081139510835DD900E2A3D88F5F70
:102A40009F4FAF4FBF4F84159505A605B705E8F218
:102A5000AA2031F40DE096D80AE094D8AA24A394D1
:102A600080E090E0A0E0B0E0EECF22ED35E08E0116
:102A70000E94631D002309F461C0088919892A890D
:102A80003B89A02F4C885D886E887F8804EB12E01C
:102A90000E9490490A2F2ED90FEB12E00E94904914
:102AA000820132D909EC12E00E94904980E00CC00A
:102AB00008E10093880701E00093890722E013E012
:102AC000082F0E9473488395A81790F70AED12E02B
:102AD0000E94904914C00EE1009388070FEF009305
:102AE000890703E000938A0723E013E0082F0E9480
:102AF00073488395A81778F782010E94580C0091BB
:102B0000F00C1091EF0C011709F0A5C980E00FC07F
:102B10000EE10093880700E00093890700E000932E
:102B20008A0723E013E0082F0E9473488395A817B3
:102B300078F782010E94580C80E0DCCF2EEC35E063
:102B40008E01C1D7002309F431C100E000935B0975
:102B500000914B090093880721E015E00EEF0E94D9
:102B6000734801E0801641F520E130E0A9010E94A0
:102B7000754B802E80E090E0E82DF0E031978E17C5
:102B80009F070CF042C0E82FF0E07196AF010E9461
:102B9000754B10E020E030E0FE017096482F50E0C9
:102BA000440F551F440F551FE40FF51F0083118379
:102BB000228333838395DFCF05E1801610F004E193
:102BC000802E20E130E0082DA9010E94814B80E099
:102BD00015C0FE017096082F10E0000F111F000FA6
:102BE000111FE00FF11F0081118122813381E82F35
:102BF000F0E07196AF010E94814B839590E0E82D43
:102C0000F0E031978E179F0724F30CE810E00E9444
:102C100090490BE50E94C20D80E004C00DE50E94C2
:102C2000C20D839590E0E82DF0E031978E179F0755
:102C3000D4F4FE017096082F10E0000F111F000F52
:102C4000111FE00FF11F008111812281338152D8C1
:102C500090E0E82DF0E032978E179F07FCF60DE22A
:102C60000E94C20DDECF0091F00C1091EF0C011705
:102C700009F098C00CE810E00E94904980E018C06C
:102C8000FE017096082F10E0000F111F000F111F9A
:102C9000E00FF11F0081118122813381102F0091FB
:102CA0004B090E941D4B26D800E20E94C20D83955D
:102CB00090E0E82DF0E031978E179F07A4F6FE0113
:102CC0007096082F10E0000F111F000F111FE00F6A
:102CD000F11F0081118122813381083CF9F00091BC
:102CE0004B09043688F100914B090E3668F504E370
:102CF00017E1FE017096282F30E0220F331F220FBC
:102D0000331FE20FF31F408151816281738150E0D4
:102D1000040F151FF80104910230B1F4FE01709602
:102D2000082F10E0000F111F000F111FE00FF11FFF
:102D30000081118122813381102F00914B090E9463
:102D40009C3A0E94840EB0CF0CEF16E1FE01709603
:102D5000282F30E0220F331F220F331FE20FF31F03
:102D6000408151816281738150E0040F151FF80189
:102D70000491023009F084CFFE017096082F10E014
:102D8000000F111F000F111FE00FF11F00811181B3
:102D900022813381102F00914B090E942C4B0E94FD
:102DA000840E82CF01E000935B0955C829EC35E021
:102DB0008E0189D6002309F447C0488859886A885B
:102DC0007B888C899D89AE89BF8900E000935B096F
:102DD000A0E04A1608F108E10093880701E000939B
:102DE000890722E013E00A2F0E947348A395F1CFD0
:102DF0000EE1009388070FEF0093890703E000932B
:102E00008A0723E013E00A2F0E947348A3954A160D
:102E100078F78C010E94580CA0E00FC00EE10093DF
:102E2000880700E00093890700E000938A0723E009
:102E300013E00A2F0E947348A3954A1678F78C0175
:102E40000E94580CA0E0E3CF25EC35E08E013BD684
:102E5000002369F0088919892A893B8900934B0965
:102E600021E030E0A9010E94814B0C942B0F20EC53
:102E700035E08E0128D6002331F42EEB35E08E01AB
:102E800022D6002321F00E940A470C942B0F29EB35
:102E900035E08E0118D6002319F03CD00C942B0F8E
:102EA00025EB35E08E010FD6002381F002E080167D
:102EB00040F0088919892A893B890E94533F0C9464
:102EC0002B0F01E00E94533F0C942B0F2EEA35E0AC
:102ED0008E01F9D5002331F42AEA35E08E01F3D5CD
:102EE000002321F0992493940C942B0F0CE810E00C
:102EF0000E94904908EE1DE00E9490490C942B0F0F
:102F000000E000935B09EF96EF96EF962796EBE0D3
:102F10000C945B4C03E319E00E94904905E519E02D
:102F20000E9490490BE719E00E94904900EA19E0DD
:102F30000E94904909EE19E00E94904900E31AE0CE
:102F40000E94904907E61AE00E9490490DE81AE0B5
:102F50000E94904908EC1AE00E94904906E01BE0AC
:102F60000E94904902E21BE00E9490490CE41BE0A1
:102F70000E94904907E81BE00E9490490CEC1BE07E
:102F80000E94904905E11CE00E94904909E51CE07F
:102F90000E94904906E91CE00E94904903EE1CE063
:102FA0000E94904908950E94514C00914B09083CA1
:102FB00009F0B9C088E10CEF1DE00E949049082F8C
:102FC0000E94070F0AE30E94C20D182F00914B09BF
:102FD0000E949C3A0E94840E839509E11EE00E94A3
:102FE0009049082F0E94070F0AE30E94C20D182F74
:102FF00000914B090E949C3A0E94840E839506E33F
:103000001EE00E949049082F0E94070F0AE30E94C9
:10301000C20D182F00914B090E949C3A0E94840E09
:103020008395839503E51EE00E949049082F0E9436
:10303000070F0AE30E94C20D182F00914B090E944E
:103040009C3A0E94840E8395839500E71EE00E94BF
:103050009049082F0E94070F0AE30E94C20D182F03
:1030600000914B090E949C3A0E94840E83950DE8C2
:103070001EE00E949049082F0E94070F0AE30E9459
:10308000C20D182F00914B090E949C3A0E94840E99
:1030900083950AEA1EE00E949049082F0E94070FBC
:1030A0000AE30E94C20D182F00914B090E949C3A1E
:1030B0000E94840E839507EC1EE00E949049082F21
:1030C0000E94070F0AE30E94C20D182F00914B09BE
:1030D0000E949C3A0E94840E839504EE1EE00E949A
:1030E0009049082F0E94070F0AE30E94C20D182F73
:1030F00000914B090E949C3A0E94840E839583950F
:1031000001E01FE00E949049082F0E94070F0AE388
:103110000E94C20D182F00914B090E949C3A0E94F8
:10312000840E839521C480E008E013E00E9490495A
:10313000082F0E94070F0CEA1DE00E949049A82F5B
:10314000B0E01596FD01E65FF74F00810E94070F82
:10315000839507E313E00E949049082F0E94070F10
:103160000CEA1DE00E949049A82FB0E01596FD01E1
:10317000E65FF74F00810E94070F839506E513E095
:103180000E949049082F0E94070F0CEA1DE00E9440
:103190009049A82FB0E01596FD01E65FF74F00813A
:1031A0000E94070F839505E713E00E949049082FBE
:1031B0000E94070F0CEA1DE00E949049A82FB0E082
:1031C0001596FD01E65FF74F00810E94070F83957A
:1031D00004E913E00E949049082F0E94070F0CEAAF
:1031E0001DE00E949049A82FB0E01596FD01E65F12
:1031F000F74F00810E94070F839503EB13E00E94B5
:103200009049082F0E94070F0CEA1DE00E94904988
:10321000A82FB0E01596FD01E65FF74F00810E94F0
:10322000070F839502ED13E00E949049082F0E943A
:10323000070F0CEA1DE00E949049A82FB0E01596F8
:10324000FD01E65FF74F00810E94070F839501EFB4
:1032500013E00E949049082F0E94070F0CEA1DE01E
:103260000E949049A82FB0E01596FD01E65FF74F48
:1032700000810E94070F839500E114E00E949049AD
:10328000082F0E94070F0CEA1DE00E949049A82F0A
:10329000B0E01596FD01E65FF74F00810E94070F31
:1032A00083950FE214E00E949049082F0E94070FB7
:1032B0000CEA1DE00E949049A82FB0E01596FD0190
:1032C000E65FF74F00810E94070F83950EE414E03C
:1032D0000E949049082F0E94070F0CEA1DE00E94EF
:1032E0009049A82FB0E01596FD01E65FF74F0081E9
:1032F0000E94070F83950DE614E00E949049082F65
:103300000E94070F0CEA1DE00E949049A82FB0E030
:103310001596FD01E65FF74F00810E94070F839528
:103320000CE814E00E949049082F0E94070F0CEA55
:103330001DE00E949049A82FB0E01596FD01E65FC0
:10334000F74F00810E94070F83950BEA14E00E945B
:103350009049082F0E94070F0CEA1DE00E94904937
:10336000A82FB0E01596FD01E65FF74F00810E949F
:10337000070F83950AEC14E00E949049082F0E94E1
:10338000070F0CEA1DE00E949049A82FB0E01596A7
:10339000FD01E65FF74F00810E94070F839509EE5C
:1033A00014E00E949049082F0E94070F0CEA1DE0CC
:1033B0000E949049A82FB0E01596FD01E65FF74FF7
:1033C00000810E94070F839508E015E00E94904954
:1033D000082F0E94070F0CEA1DE00E949049A82FB9
:1033E000B0E01596FD01E65FF74F00810E94070FE0
:1033F000839507E215E00E949049082F0E94070F6D
:103400000CEA1DE00E949049A82FB0E01596FD013E
:10341000E65FF74F00810E94070F839506E415E0F1
:103420000E949049082F0E94070F0CEA1DE00E949D
:103430009049A82FB0E01596FD01E65FF74F008197
:103440000E94070F839505E615E00E949049082F1A
:103450000E94070F0CEA1DE00E949049A82FB0E0DF
:103460001596FD01E65FF74F00810E94070F8395D7
:1034700004E815E00E949049082F0E94070F0CEA0B
:103480001DE00E949049A82FB0E01596FD01E65F6F
:10349000F74F00810E94070F839503EA15E00E9411
:1034A0009049082F0E94070F0CEA1DE00E949049E6
:1034B000A82FB0E01596FD01E65FF74F00810E944E
:1034C000070F839502EC15E00E949049082F0E9497
:1034D000070F0CEA1DE00E949049A82FB0E0159656
:1034E000FD01E65FF74F00810E94070F839501EE13
:1034F00015E00E949049082F0E94070F0CEA1DE07A
:103500000E949049A82FB0E01596FD01E65FF74FA5
:1035100000810E94070F83950EEE12E00E949049F1
:103520000E94F30E00E016E00E949049082F0E94CE
:10353000070F0CEA1DE00E949049A82FB0E01596F5
:10354000FD01E65FF74F00810E94070F83950CE2B3
:1035500016E00E949049082F0E94070F0CEA1DE018
:103560000E949049A82FB0E01596FD01E65FF74F45
:1035700000810E94070F83950BE416E00E9490499A
:10358000082F0E94070F0CEA1DE00E949049A82F07
:10359000B0E01596FD01E65FF74F00810E94070F2E
:1035A00083950AE616E00E949049082F0E94070FB3
:1035B0000CEA1DE00E949049A82FB0E01596FD018D
:1035C000E65FF74F00810E94070F839509E816E038
:1035D0000E949049082F0E94070F0CEA1DE00E94EC
:1035E0009049A82FB0E01596FD01E65FF74F0081E6
:1035F0000E94070F839508EA16E00E949049082F61
:103600000E94070F0CEA1DE00E949049A82FB0E02D
:103610001596FD01E65FF74F00810E94070F839525
:1036200007EC16E00E949049082F0E94070F0CEA51
:103630001DE00E949049A82FB0E01596FD01E65FBD
:10364000F74F00810E94070F839506EE16E00E9457
:103650009049082F0E94070F0CEA1DE00E94904934
:10366000A82FB0E01596FD01E65FF74F00810E949C
:10367000070F839505E017E00E949049082F0E94EC
:10368000070F0CEA1DE00E949049A82FB0E01596A4
:10369000FD01E65FF74F00810E94070F839504E26A
:1036A00017E00E949049082F0E94070F0CEA1DE0C6
:1036B0000E949049A82FB0E01596FD01E65FF74FF4
:1036C00000810E94070F839503E417E00E94904950
:1036D000082F0E94070F0CEA1DE00E949049A82FB6
:1036E000B0E01596FD01E65FF74F00810E94070FDD
:1036F000839502E617E00E949049082F0E94070F69
:103700000CEA1DE00E949049A82FB0E01596FD013B
:10371000E65FF74F00810E94070F839501E817E0ED
:103720000E949049082F0E94070F0CEA1DE00E949A
:103730009049A82FB0E01596FD01E65FF74F008194
:103740000E94070F839500EA17E00E949049082F16
:103750000E94070F0CEA1DE00E949049A82FB0E0DC
:103760001596FD01E65FF74F00810E94070F8395D4
:103770000FEB17E00E949049082F0E94070F0CEAF8
:103780001DE00E949049A82FB0E01596FD01E65F6C
:10379000F74F00810E94070F83950EED17E00E94FE
:1037A0009049082F0E94070F0CEA1DE00E949049E3
:1037B000A82FB0E01596FD01E65FF74F00810E944B
:1037C000070F83950DEF17E00E949049082F0E9484
:1037D000070F0CEA1DE00E949049A82FB0E0159653
:1037E000FD01E65FF74F00810E94070F83950CE112
:1037F00018E00E949049082F0E94070F0CEA1DE074
:103800000E949049A82FB0E01596FD01E65FF74FA2
:1038100000810E94070F83950BE318E00E949049F6
:10382000082F0E94070F0CEA1DE00E949049A82F64
:10383000B0E01596FD01E65FF74F00810E94070F8B
:1038400083950AE518E00E949049082F0E94070F0F
:103850000CEA1DE00E949049A82FB0E01596FD01EA
:10386000E65FF74F00810E94070F839509E718E094
:103870000E949049082F0E94070F0CEA1DE00E9449
:103880009049A82FB0E01596FD01E65FF74F008143
:103890000E94070F839508E918E00E949049082FBD
:1038A0000E94070F0CEA1DE00E949049A82FB0E08B
:1038B0001596FD01E65FF74F00810E94070F839583
:1038C00007EB18E00E949049082F0E94070F0CEAAE
:1038D0001DE00E949049A82FB0E01596FD01E65F1B
:1038E000F74F00810E94070F839506ED18E00E94B4
:1038F0009049082F0E94070F0CEA1DE00E94904992
:10390000A82FB0E01596FD01E65FF74F00810E94F9
:10391000070F839505EF18E00E949049082F0E9439
:10392000070F0CEA1DE00E949049A82FB0E0159601
:10393000FD01E65FF74F00810E94070F839504E1C8
:1039400019E00E949049082F0E94070F0CEA1DE021
:103950000E949049A82FB0E01596FD01E65FF74F51
:1039600000810E94070F8395E4E00C94624C9A93C7
:103970008A93902F80E000915909109158090117FE
:10398000D1F340E050E060E070E0009159091091FF
:1039900058090117A1F48A019B01A801B9014F5FE1
:1039A0005F4F6F4F7F4F013EE3E91E07E4E02E07B4
:1039B000E0E03E0750F3082F899199910895009116
:1039C000590910E0F801E857F94F0081E9E5F9E0FD
:1039D000108113951083282F30E0F901E65FF74F2F
:1039E0000083992341F0082F10E0F801E65FF74FBC
:1039F00000810E94C20D8395C4CF0E94514C902F2C
:103A0000A12FB22FA0938807B093890700EF0093EE
:103A10008A0705E500938B070FE000938C070AEAFD
:103A200000938D0726E01DE0092F0E94F847802FA4
:103A300000915B09002349F00CE810E00E949049D6
:103A4000282F0EEB18E00E9449480AE010E00E947F
:103A5000580C1A2F092F0E941D4B0B1711F401E06F
:103A600001C000E0E4E00C94624C0F3130F410E04F
:103A7000F801E35AF64F00810895043650F00E36EF
:103A800040F410E004561040F801E358F64F00816E
:103A9000089500E00895A80100E001C00395083CE6
:103AA00088F410E0F901E00FF11F608110E0FA01E5
:103AB000E00FF11F608310E0F901E00FF11F1081AA
:103AC000112361F70895A80100E010E0FA01E00F6A
:103AD000F11F608110E0F901E00FF11F1081611703
:103AE00091F4039510E0FA01E00FF11F108111230A
:103AF00039F410E0F901E00FF11F1081112321F0DA
:103B0000093C18F3089500E008950E944E4CD90135
:103B1000CA01442401C043945524FC01E40DF51D61
:103B200020812032C1F32CE3421608F041C0552415
:103B3000FC01E40DF51D20812223D1F120E021C0FC
:103B40005524FC01E40DF51D3081313670F055240B
:103B5000FC01E40DF51D30813B3738F45524FC01A0
:103B6000E40DF51D30813F7530835524FC01E40DD3
:103B7000F51D408130E0F801E20FF31F40832395EB
:103B800043945524FC01E40DF51D3081303350F091
:103B90005524FC01E40DF51D30813B3718F430E16C
:103BA000431670F240E030E0F801E20FF31F40836B
:103BB000E02FF12F0081002311F400E0A6C066245D
:103BC0009EC043945524FC01E40DF51D0081003294
:103BD000C1F35524FC01E40DF51D0081002319F407
:103BE0006394062D92C000E010E020E030E0462D06
:103BF00050E0440F551F440F551FFD01E40FF51F02
:103C0000008311832283338342C0062D10E0000F0E
:103C1000111F000F111FFD01E00FF11F0081118125
:103C2000228133814AE050E060E070E00E94D44B92
:103C3000462D50E0440F551F440F551FFD01E40F62
:103C4000F51F00831183228333835524FC01E40D87
:103C5000F51D008110E000531040212F220F220B90
:103C6000322F462D50E0440F551F440F551FFD01C4
:103C7000E40FF51F4081518162817381400F511F14
:103C8000621F731F408351836283738343940CE3E9
:103C90004016A0F55524FC01E40DF51D008100231C
:103CA00021F402E0600E062D30C05524FC01E40D25
:103CB000F51D00810B33E1F05524FC01E40DF51DE9
:103CC00000810A33A9F05524FC01E40DF51D0081A3
:103CD0000C3271F05524FC01E40DF51D00810E320B
:103CE00039F05524FC01E40DF51D0081003281F40A
:103CF00000E25524FC01E40DF51D008363940EE100
:103D0000601608F45FCF6394062DE7E00C945F4CD7
:103D100000915209002309F478CF5524FC01E40DE9
:103D2000F51D0081003308F446C05524FC01E40D64
:103D3000F51D00810A33F8F5062D10E0000F111F64
:103D4000000F111FFD01E00FF11F00811181228181
:103D5000338144E00E94F04B462D50E0440F551F44
:103D6000440F551FFD01E40FF51F008311832283CB
:103D700033835524FC01E40DF51D008110E0005350
:103D80001040212F220F220B322F462D50E0440FDE
:103D9000551F440F551FFD01E40FF51F4081518150
:103DA00062817381400F511F621F731F40835183D3
:103DB000628373836BCF5524FC01E40DF51D0081F4
:103DC000013408F463CF5524FC01E40DF51D008196
:103DD0000B3708F05BCF5524FC01E40DF51D008185
:103DE0000F750083062D10E0000F111F000F111F2B
:103DF000FD01E00FF11F008111812281338144E038
:103E00000E94F04B462D50E0440F551F440F551FA4
:103E1000FD01E40FF51F00831183228333835524B2
:103E2000FC01E40DF51D008110E007531040212F27
:103E3000220F220B322F462D50E0440F551F440F06
:103E4000551FFD01E40FF51F40815181628173818F
:103E5000400F511F621F731F40835183628373831E
:103E600015CF0E94514CC801A22FB1E016C008E046
:103E70000E94C20D00E20E94C20D08E00E94C20D25
:103E80000A2FA02FAA95002391F721EB3DE08C018A
:103E900002DEA02F8C010E94E60EBB23A9F10E9436
:103EA000F30E102F1050C9F31A9551F3175099F0D3
:103EB000125029F0135019F01E5079F319C000E088
:103EC000B0E0FC01EA0FFB1F00839C0101EB1DE049
:103ED000E2DD01E01AC0A13000F3AA9508E00E94DB
:103EE000C20D00E20E94C20D08E00E94C20DD5CFB3
:103EF000AC3398F62A2F30E0FC01E20FF31F008369
:103F00000E94C20DA395C9CF00E0E4E00C94624C7E
:103F10000E94514C902F812F983050F5883040F5F9
:103F2000092F10E00F5F1F4F40E450E00E94934BB9
:103F3000D801082F10E00F5F1F4F40E450E00E94AF
:103F4000934B20E011C0422F50E0400F511FFA0167
:103F5000E853F64F3081422F50E04A0F5B1FFA01C1
:103F6000E853F64F30832395203468F3092F03D0AC
:103F7000E4E00C94624C9A938A93902F973011F45A
:103F800090E001C0939580E007C0182F092F27D239
:103F9000182F092F2BD183958F31B8F31FE1092FEB
:103FA0001ED21FE1092FD3D0F801E853F64F00814C
:103FB0000E947A0E10E2092F12D210E2092FC7D008
:103FC000F801E853F64F00810E947A0E8991999189
:103FD0000895005049F00A9561F00A9579F00A9524
:103FE00091F00A95A9F008950DEB14E10E94904913
:103FF000089501ED14E10E94904908950FED14E138
:104000000E949049089502EF14E10E94904908959A
:1040100002E015E10E94904908959A938A93802FB7
:10402000912FE9EFF5E11491E0EFF5E104910E94A1
:10403000AB2E22E0082F10E00E948D0EEAEFF5E192
:104040001491E1EFF5E104910E94AB2E22E0092FDB
:1040500010E00E948D0EEBEFF5E11491E2EFF5E137
:1040600004910E94AB2E192F082F71D00E94840E4C
:104070008991999108958A93E3EFF5E11491EAEE1D
:10408000F5E104910E94AB2E80E004C000E20E94A2
:10409000C20D83958634D0F3E3EFF5E11491EAEE97
:1040A000F5E104910E94AB2E899108959A938A9329
:1040B0009091DC0980E00CC0182F0091ED0D039564
:1040C0008ED108E00E94C20D00E20E94C20D8395CD
:1040D0008F3190F380E00BC0182F092F03957FD10B
:1040E00008E00E94C20D0CE70E94C20D83958F313B
:1040F00098F39093ED0DE7EFF5E11491EEEEF5E115
:1041000004910E94AB2E092F0E947A0E89919991F9
:104110000895093031F4133020F0143110F401E027
:104120000895083021F41F3110F401E0089508309B
:1041300030F4103211F01F3111F401E0089508300D
:1041400020F4103210F402E0089500E00895682F82
:10415000202F812F222371F48F3138F4082F10E0A3
:10416000000F111F00501E4F39C0082F10E0015ED4
:104170001D4F34C08F3149F4022F10E040E450E06D
:104180000E94934B025C1F4F29C0803249F4022FDA
:1041900010E040E450E00E94934B015C1F4F1EC0B2
:1041A000283029F4082F10E0005E1F4F17C0293077
:1041B00029F4082F10E0055F1F4F10C0022F10E0F8
:1041C0000150104040E450E00E94934B980102E0FF
:1041D000809F8001020F131F005C1F4F003422E0FC
:1041E000120710F000E010E0862F08959A938A934A
:1041F000902F812F8F3108F042C0182F092FA7DF91
:10420000F801E853F64F20813181203004E0300777
:1042100048F0182F092F9BDFF801E853F64F018172
:1042200007FF0BC0182F092F92DFF801E853F64F54
:10423000008111810E94840E22C0182F092F87DF70
:10424000F801E853F64F018105FF0DC00FE30E940E
:10425000C20D0FE30E94C20D0FE30E94C20D0FE3D7
:104260000E94C20D0CC00DE20E94C20D0DE20E9420
:10427000C20D0DE20E94C20D0DE20E94C20D899195
:10428000999108959A938A930091CC0C002351F050
:1042900000E09FDE0E94F30E093521F0093711F08E
:1042A00000E05CC0EAECFCE00081118120E030E03D
:1042B00040E052E060E070E00E94D44BA801B901F8
:1042C000405050426F4F7F4F10E080E090E017C0A9
:1042D0000C0122243324040E151E261E371EF00165
:1042E000322D3BBF069000E00BBFFC01E853F64FB8
:1042F0000082FC01E853F64F0081100F01968030D8
:1043000002E0900728F300E015C0202F30E0F9010B
:10431000E35AF64F2081222361F440E050E422E08A
:10432000029F900120503E4FF901E853F64F408321
:10433000518303950F3148F31F3F21F40091DC09AD
:10434000083008F00ED000E00093CC0C0091DF099B
:10435000053018F000E00093DF0901E089919991A0
:1043600008953B2F2A2FE0E0F0E006C000E0DF01D7
:10437000A853B64F0C933196E03200E0F007B0F34B
:10438000E0E2F0E006C005E5DF01A853B64F0C936C
:104390003196E03400E0F007B0F3E0E4F0E009C06B
:1043A00000E010E4DF01A853B64F0D931C93119762
:1043B0003296E03002E0F00798F300E00093DC0969
:1043C00001E00093D70900E20093DE0900E20093C8
:1043D000E00900E00093D509A22FB32F08959A9326
:1043E0008A936297602F212FCE010896EAE4F9E9BB
:1043F00030E08C014AE050E00E94344CCE01E4E50C
:10440000F9E930E08C0148E050E00E94344C203261
:1044100011F02F3151F42395122FFE0170E0E60FB9
:10442000F71F00810E94AB2E10C02F3158F4239546
:10443000122FFE01389670E0E60FF71F00810E94F0
:10444000AB2E03C001E20E94C20D62968991999140
:1044500008958A93802F03C000E20E94C20D082FA6
:10446000802F8A950023C1F7899108950E94524CAC
:1044700080E005C00CE810E00E94904983958C33E1
:10448000C8F311E001E00E94AB2E0EE11FE00E9494
:10449000904908E31FE00E94904907E2DADF03E554
:1044A0001FE00E94904900E61FE00E94904907E249
:1044B000D0DF0BE71FE00E94904902E81FE00E9456
:1044C000904907E2C6DF0DE91FE00E9490490BEA20
:1044D0001FE00E94904907E2BCDF06EC1FE00E944B
:1044E000904904ED1FE00E94904907E2B2DF0FEE11
:1044F0001FE00E9490490DEF1FE00E94904907E2E3
:10450000A8DF08E110E10E94904906E210E10E9454
:10451000904907E29EDF01E410E10E9490490FE418
:1045200010E10E94904907E294DF0AE610E10E9440
:10453000904908E710E10E94904907E28ADF03E909
:1045400010E10E94904901EA10E10E94904907E2BF
:1045500080DF0CEB10E10E9490490AEC10E10E9410
:10456000904907E276DF05EE10E10E94904903EFE3
:1045700010E10E94904907E26CDF0EE011E10E9419
:1045800090490CE111E10E94904907E262DF07E3E4
:1045900011E10E94904905E411E10E94904907E26F
:1045A00058DF00E611E10E9490490EE611E10E94F9
:1045B000904907E24EDF09E811E10E94904907E9BE
:1045C00011E10E94904907E244DF02EB11E10E94F1
:1045D000904900EC11E10E94904907E23ADF0BEDAF
:1045E00011E10E94904909EE11E10E94904907E211
:1045F00030DF04E012E10E94904902E112E10E94E2
:10460000904907E226DF0DE212E10E9490490BE398
:1046100012E10E94904906E512E10E94904901E7EB
:1046200012E10E9490490CE812E10E94904907EAC9
:1046300012E10E94904902EC12E10E9490490DEDB6
:1046400012E10E94904908EF12E10E94904903E1B3
:1046500013E10E9490490EE213E10E94904909E49F
:1046600013E10E94904904E613E10E9490490FE78C
:1046700013E10E949049EAECFCE000811181012BDA
:1046800029F40FE114E10E94904904C000ED13E108
:104690000E9490490EE614E10E94904980E001C01A
:1046A00083958132F8F490E006C0A23019F4182FF7
:1046B000092F9CDD9395933198F7182F092F29DD49
:1046C000A02FAA23B9F3182F092F89DEA13069F78B
:1046D000182F092F3CDDF801E853F64F00810E94A6
:1046E0007A0EE8CFE3DCE4EFF5E11491EBEEF5E1CF
:1046F00004910E94AB2E08EC19E00E94E60EE5EF53
:10470000F5E11491ECEEF5E104910E94AB2EEAEC98
:10471000FCE0008111810E94840EE6EFF5E1149126
:10472000EDEEF5E104910E94AB2EEAECFCE0008195
:10473000118120E030E040E052E060E070E00E9453
:10474000D44B005010422F4F3F4F0E94D50EE3E054
:104750000C94634C0E94484CEF97EA97DA95BE019F
:1047600064527F4FECE5F9E930E08B0141E250E023
:104770000E94344CA0E0BA2FBA2ECA2E24EF3FE09C
:10478000A9010E94754B053511F40C94C82D1A2F00
:104790000B2F43DC1A2F0B2F22DE9090DC090091A7
:1047A0005209002319F000E1A02E02C00AE0A02E59
:1047B0000E94F30E902F9B31D9F50E94F30E902F9B
:1047C0009B3519F40E94F30E902F943421F4BB23EF
:1047D00089F0BA950FC0933411F4B3950BC091349E
:1047E00021F4AA2339F0AA9505C0923419F4A03215
:1047F00008F4A395FE01E452FF4F0A2F10E0E00FEA
:10480000F11F00810B1738F4FE01E452FF4FB0E0B6
:10481000EA0FFB1FB081BC1521F4AB1511F40C9409
:10482000622E1A2F0B2FF9DBCB2EBA2E0C94622E90
:10483000903209F044C01A2F0B2F6BDC023011F0BC
:104840000C94622E80E090E21A2F0B2F80DCF8018E
:10485000E853F64F0081118108271927008311833F
:10486000BB2329F58A2F02E0809F800100501E4F54
:10487000F801E853F64F018105FD16C090E0FC01F8
:10488000E35AF64F0081002379F014E2082F0E94CA
:104890007F2E22E0829F20E0020E22E0121EF00115
:1048A000E853F64F008311830A2F0E9445381A2FD0
:1048B0000B2F9CDC01E00093CC0C0C94622E9D35F8
:1048C00009F04CC01A2F0B2F8ADD1A2F0B2F21DC79
:1048D0000130B9F41A2F0B2F3ADCF801E853F64FE8
:1048E0000081039500831A2F0B2F31DCF801E85368
:1048F000F64F00810E947A0E01E00093CC0C0C94DC
:10490000622E023011F00C94622E1A2F0B2F1FDC36
:10491000F801E853F64F008111810F7F13700F3FAC
:1049200023E0120711F40C94622E1A2F0B2F0FDCC8
:10493000F801E853F64F008111810F5F1F4F00838C
:1049400011831A2F0B2F52DCBB2319F40A2F0E945C
:10495000453801E00093CC0C0C94622E9B3509F095
:104960004AC01A2F0B2F3BDD1A2F0B2FD2DB013041
:10497000B9F41A2F0B2FEBDBF801E853F64F008147
:104980000A9500831A2F0B2FE2DBF801E853F64F4C
:1049900000810E947A0E01E00093CC0C0C94622EF0
:1049A000023011F00C94622E1A2F0B2FD0DBF8017D
:1049B000E853F64F008111810F7F1370012B11F422
:1049C0000C94622E1A2F0B2FC2DBF801E853F64F1E
:1049D0000081118101501040008311831A2F0B2F89
:1049E00005DCBB2319F40A2F0E94453801E000932F
:1049F000CC0C0C94622E9D3709F050C01A2F0B2F4F
:104A000088DB0130B9F41A2F0B2FA1DBF801E85332
:104A1000F64F00810A0D00831A2F0B2F98DBF80147
:104A2000E853F64F00810E947A0E01E00093CC0C0F
:104A30000C94622E023011F00C94622E1A2F0B2F60
:104A400086DBF801E853F64F008111810F7F137068
:104A50002FEF33E04A2D50E0241B350B02171307CC
:104A600010F00C94622E8A2D90E01A2F0B2F6FDB22
:104A7000F801E853F64F00811181080F191F0083D8
:104A800011831A2F0B2FB2DBBB2319F40A2F0E94BC
:104A9000453801E00093CC0C0C94622E9B3709F052
:104AA0004CC01A2F0B2F35DB0130B9F41A2F0B2F06
:104AB0004EDBF801E853F64F00810A1900831A2FE4
:104AC0000B2F45DBF801E853F64F00810E947A0E68
:104AD00001E00093CC0C0C94622E023011F00C9487
:104AE000622E1A2F0B2F33DBF801E853F64F0081AB
:104AF00011810F7F13702A2D30E00217130710F475
:104B00000C94622E8A2D90E01A2F0B2F20DBF801D7
:104B1000E853F64F00811181081B190B00831183A4
:104B20001A2F0B2F63DBBB2319F40A2F0E94453881
:104B300001E00093CC0C0C94622E9DDA903360F06F
:104B40009B3750F4092F0E94C20D98A721E08E01D7
:104B5000085D1F4F86D905C020E08E01085D1F4FFC
:104B600080D900E00883AE01485D5F4F9E012C595B
:104B70003F4F8E010E94851D902F992311F40C94B4
:104B8000622E23E935E08E010E94631D002351F05F
:104B900001E000935209A0E0BA2F1A2F0B2F3DDA43
:104BA0000C94622E2FE835E08E010E94631D0023D5
:104BB00051F000E000935209A0E0BA2F1A2F0B2FFA
:104BC0002CDA0C94622E2BE336E08E010E94631DDA
:104BD000002341F04BDCA0E0BA2F1A2F0B2F1DDA77
:104BE0000C94622E27E336E08E010E94631D0023A1
:104BF00039F427ED35E08E010E94631D002391F00A
:104C0000E3EFF5E11491EAEEF5E104910E94AB2E99
:104C10000E94170F2BDCA0E0BA2F1A2F0B2FFDD903
:104C20000C94622E22E336E08E010E94631D002365
:104C3000B1F0933021F002E0CCD90C94622EFE0149
:104C4000FF9605A116A127A130A5B02FFE01FF9662
:104C500001A512A523A534A5A02F0C94622E2DE248
:104C600036E08E010E94631D002339F42BE236E00A
:104C70008E010E94631D002341F1EAECFCE02081DB
:104C800031812F3700E03007E8F4EAECFCE00081E6
:104C900011810F5F1F4F00831183F4DA002341F06D
:104CA000E5DBA0E0BA2F1A2F0B2FB7D90C94622E98
:104CB000EAECFCE000811181015010400083118377
:104CC0000C94622E01E085D9FDC724E236E08E0106
:104CD0000E94631D002339F422E236E08E010E9417
:104CE000631D002321F1EAECFCE000811181012B1E
:104CF000D9F0EAECFCE00081118101501040008302
:104D00001183C0DA002339F0B1DBA0E0BA2F1A2FEB
:104D10000B2F83D9D7C7EAECFCE0008111810F5F2C
:104D20001F4F00831183CEC701E053D9CBC72DE1BC
:104D300036E08E010E94631D002339F42BE136E03A
:104D40008E010E94631D002399F1923019F002E058
:104D500040D9B8C7FE01FF9605A116A127A130A52D
:104D6000003840E0140740E0240740E03407E8F44E
:104D7000EAECFCE080819181FE01FF9605A116A17D
:104D800027A130A5EAECFCE0008311837BDA002345
:104D900039F06CDBA0E0BA2F1A2F0B2F3ED992C747
:104DA000EAECFCE0808391838DC701E012D98AC7C9
:104DB00026E136E08E010E94631D0023D1F192307E
:104DC00019F002E006D97EC7FE01FF9605A116A1E3
:104DD00027A130A5003840E0140740E0240740E058
:104DE000340720F5EAECFCE080819181FE01FF961A
:104DF00005A116A127A130A5EAECFCE000831183F0
:104E000041DA002371F0EAECFCE0808391832EDB31
:104E1000A0E0BA2F1A2F0B2F00D901E00093CC0C81
:104E200051C7EAECFCE0808391834CC701E0D1D804
:104E300049C728E436E08E010E94631D0023E1F09B
:104E40000091CC0C002389F000E0C3D80E94F30E3F
:104E5000902F993519F0993709F034C704E110E023
:104E60000E94580C08E001BD2DC704E110E00E942B
:104E7000580C08E001BD26C721E136E08E010E94F2
:104E8000631D002319F10AE30E94C20D20E08E0188
:104E9000085D1F4F0E94311F002361F000E00DAB41
:104EA0009E01285D3F4F08EC19E00E944B1D01E078
:104EB0000093CC0CE4EFF5E11491EBEEF5E10491F5
:104EC0004AD708EC19E00E94E60EFCC62EE036E058
:104ED0008E010E94631D002309F482C09130A9F560
:104EE00080E08F3108F0EEC602E0809F00E0000E07
:104EF00002E0101EF001E853F64F018105FF23C0C8
:104F000090E0FC01E35AF64F00810023E1F021E03C
:104F100018E1082F0E94424B14E2082FF0D622E03D
:104F2000829F20E0020E22E0121EF001E853F64FAD
:104F300000831183082F0E944538182F00E04FDAB4
:104F4000182F00E053D98395CCCF44245524E92F62
:104F5000F0E031974E165F060CF0B4C6FE01EC5936
:104F6000FF4F042D10E0000F111F000F111FE00F65
:104F7000F11F0081118122813381802F02E0809F07
:104F800000E0000E02E0101EF001E853F64F018130
:104F900005FF24C0082F10E0F801E35AF64F008106
:104FA0000023E1F021E018E1082F0E94424B14E2B7
:104FB000082FA5D622E0829F20E0020E22E0121EDA
:104FC000F001E853F64F00831183082F0E94453803
:104FD000182F00E004DA182F00E008D94394B6CF68
:104FE0002AE036E08E010E94631D002309F460C0B0
:104FF000913021F580E08F3108F064C690E0FC012B
:10500000E35AF64F00810023B9F020E018E1082FA1
:105010000E94424B02E0809F00E0000E02E0101E62
:10502000F001E853F64F018100620183182F00E080
:10503000D6D9182F00E0DAD88395DDCF4424552443
:10504000E92FF0E031974E165F060CF03BC6FE01EB
:10505000EC59FF4F042D10E0000F111F000F111F1E
:10506000E00FF11F0081118122813381802F082FF1
:1050700010E0F801E35AF64F00810023B9F020E078
:1050800018E1082F0E94424B02E0809F00E0000ED2
:1050900002E0101EF001E853F64F01810062018327
:1050A000182F00E09CD9182F00E0A0D84394C7CF58
:1050B00022E036E08E010E94631D002309F448C0FF
:1050C0000091F00C1091EF0C011709F0FBC508ECF2
:1050D00010E00E94580C0E943B20E3EFF5E1149190
:1050E000EAEEF5E1049137D612E205E60E941D4B87
:1050F0000E947A0E00E20E94C20D13E205E60E94B1
:105100001D4B0E947A0E00E20E94C20D14E205E6D9
:105110000E941D4B0E947A0E0CE20E94C20D12E208
:1051200006E60E941D4B0E947A0E00E20E94C20D0C
:1051300013E206E60E941D4B0E947A0E00E20E94D6
:10514000C20D14E206E60E941D4B0E947A0EB8CFF3
:1051500023E836E08E010E94631D002339F421E824
:1051600036E08E010E94631D0023C1F0FE01FF9610
:1051700005A116A127A130A5923021F002E00E94DE
:10518000E91FA0C5083020F004E00E94E91F9AC57D
:105190000093DC0901E00093CC0C94C52CE736E0C9
:1051A0008E010E94631D002399F1933021F002E0EB
:1051B0000E94E91F87C5FE01FF9605A116A127A140
:1051C00030A5802FFE01FF9601A512A523A534A5C9
:1051D000902F983010F4883020F004E00E94E91FEE
:1051E00071C50AE30E94C20D082F0E947A0E0DE2DB
:1051F0000E94C20D0EE30E94C20D092F0E947A0E7A
:10520000182F092F0E94881F01E00093CC0C5AC56B
:1052100028E735E08E010E94631D002341F423E757
:1052200035E08E010E94631D002309F488C093308D
:1052300020F002E00E94E91F45C5913019F4009169
:10524000DC0906C0FE01FF9605A116A127A130A525
:10525000073020F004E00E94E91F34C5EAECFCE0CE
:1052600020813181232B41F41091DC09133020F08F
:1052700004E00E94E91F26C5923039F417E00E942D
:10528000881F01E00093CC0C19C09130A1F400916B
:10529000DC09073080F417E00091DC090E94881FC8
:1052A000E8ECF9E004890395048B0E94562001E0A4
:1052B0000093CC0C03C004E00E94E91FEAECFCE080
:1052C00000811181012B09F0FDC40091DC0901303E
:1052D00029F00091DC09023009F0F4C400E410E088
:1052E00020E830E040EC50E080E01EC062E0869FA5
:1052F000020E131EF001E853F64F2080318062E069
:10530000869F000E111EF001E853F64F60817181F7
:10531000261A370A62E0869F040E151EF001E85334
:10532000F64F2082318283958F3100F30E943B201B
:1053300003E00E94E91F02E00E94BB1FC3C425E7EF
:1053400036E08E010E94631D002339F42BEF35E017
:105350008E010E94631D0023E9F1923029F5FE01C0
:10536000FF9605A116A127A130A5802F873020F038
:1053700004E00E94E91FA6C40091DC09801770F4C4
:10538000E8ECF9E004890A95048B0E94562006C0D7
:10539000182F1395082F0E94881F83958630C0F31D
:1053A00001E00093CC0C8EC4913009F08BC40091C5
:1053B000DC09013058F0E8ECF9E004890A95048B27
:1053C0000E94562001E00093CC0C7CC404E00E94B3
:1053D000E91F78C42EE636E08E010E94631D00238B
:1053E00039F42CE636E08E010E94631D002389F11A
:1053F000FE01FF9605A116A127A130A5802F9230AE
:1054000021F002E00E94E91F5DC4873020F004E033
:105410000E94E91F57C406E0402E06C0142D1A95BD
:10542000042D0E94881F4A948415C0F317E0082FAA
:105430000E94881F0091DC09801738F4E8ECF9E03D
:1054400004890395048B0E94562001E00093CC0C44
:1054500039C425EB35E08E010E94631D002379F0ED
:10546000923048F0FE01FF9605A116A127A130A5B4
:105470000E94533F27C401E00E94533F23C42AE403
:1054800035E08E010E94631D002341F428E435E0DD
:105490008E010E94631D002309F461C0FE01FF9686
:1054A00005A116A127A130A5402E923021F002E0DF
:1054B0000E94E91F07C407E0401620F004E00E94A4
:1054C000E91F00C499E580E01DC0082F10E0F80135
:1054D000E35AF64F00810023A1F0042D10E040E4D0
:1054E00050E00E94934B22E0829F000E111E00E4C8
:1054F000000E00E0101EF001E853F64F018106FD9A
:105500009EE483958F3108F30091DC09401640F04A
:10551000993531F400E00E94E91F0E94F30E902FAC
:10552000993519F0993709F0CDC3E8EFF5E11491F9
:10553000EFEEF5E104910FD4042D0E947A0E07E0FE
:105540000E94BB1F142D07E00E94881F80E08F314E
:1055500008F0B8C3082F0E9445388395F8CF27E696
:1055600036E08E010E94631D002309F4B0C0EAEC0E
:10557000FCE040805180913061F4EAECFCE0008175
:10558000118120E030E0FE01FF9605A316A327A3BA
:1055900030A7E7EAFDE020813181273302E03007C0
:1055A00038F023E333E012E20EEF0E944A4B06C0CC
:1055B0002FEF33E012E20EEF0E944A4B00E010E0C2
:1055C000EAECFCE00083118380E00CC022E0829FC3
:1055D00020E0020E22E0121EF001E853F64F008395
:1055E000118383958F3100F590E0FC01E35AF64F6B
:1055F00000810023B1F318E1082F0E941D4B0130F8
:1056000021F41EE1082F7BD303C014E2082F77D3C7
:10561000003020E41207D1F60DED1DE00E94904904
:10562000082F0E947A0EDDCFEAECFCE04082518226
:10563000FE01FF9605A116A127A130A59CD411C09B
:105640000091F00C1091EF0C011759F00E94F30E2D
:105650000B3139F401E00093CD0C05EF1DE00E9401
:1056600090490091CF0C002359F700E115E10E9409
:10567000904904EF11E00E94580C80E00CC022E039
:10568000829F20E0020E22E0121EF001E853F64F46
:105690000083118383958F31B0F490E0FC01E35ACD
:1056A000F64F00810023B1F31EE1082F28D300300C
:1056B00020E4120721F70DED1DE00E949049082F0C
:1056C0000E947A0EE7CF07E00E94BB1FFBC223E6D1
:1056D00036E08E010E94631D002309F457C092300A
:1056E00051F4FE01FF9605A116A127A130A50030B7
:1056F00024E0120720F002E00E94E91FE3C21A2F03
:105700000B2F0E94EF211A2F0B2F0E9489200130AE
:10571000E9F4FE01FF9605A116A127A130A5802F6F
:105720001A2F0B2F0E94A720F801E853F64F808311
:105730001A2F0B2F0E94A720F801E853F64F008183
:105740000E947A0E01E00093CC0CBCC2023009F03A
:10575000B9C2FE01FF9605A116A127A130A5C80177
:105760001A2F0B2F0E94A720F801E853F64F8083D1
:1057700091831A2F0B2F0E94F620BB2319F40A2FB6
:105780000E94453801E00093CC0C9CC22CE536E029
:105790008E010E94631D002341F42AE536E08E014C
:1057A0000E94631D002309F443C1BE01605F7F4F67
:1057B000EDE7F9E930E08B0148E150E00E94344C1C
:1057C000923071F4FE01FF9605A116A127A130A524
:1057D000073040E0140740E0240740E0340720F0A1
:1057E00002E00E94E91F6EC201E00093CC0CFE01B2
:1057F000FF9605A116A127A130A5102F07E00E9452
:10580000881F40E452EE60E070E080E03AC002E0C1
:10581000809F8001212F220F220B322F040F151F92
:10582000261F371F0F5F1F4F2F4F3F4FF801322F9B
:105830003BBF069000E00BBF302C222402E0809F8B
:105840008001212F220F220B322F040F151F261F3C
:10585000371FF801322F3BBF0690202D00E00BBF11
:1058600030E0220D331D2F7F3370FE01E55CFE4FCB
:10587000082F10E0000F111FE00FF11F208331836C
:1058800083958F3120F2FE01FF9605A116A127A175
:1058900030A540E450E00E94934B005C1F4F80E035
:1058A00026C022E0829F000E111E21E0020E20E0A1
:1058B000121EF001E853F64F508140E022E0829F33
:1058C000000E111EF001E853F64F208130E0240F46
:1058D000351F2F7F3370FE01E350FF4F482F50E0FC
:1058E000440F551FE40FF51F2083318383958F31BB
:1058F000C0F280E068C0FE01E55CFE4F082F10E0BA
:10590000000F111FE00FF11F208131812F7F3370B5
:105910008E0103501F4FFE01709690E0E80FF91FB3
:10592000408150E0440F551F040F151FE02FF12F49
:10593000008111810F7F1370201B310B8E01055CDC
:105940001E4FFE01709690E0E80FF91F408150E075
:10595000440F551F040F151FE02FF12F00811181F7
:105960000F7F1370020F131F22E0829F20E0020EB0
:1059700022E0121EF001E853F64F008311838E01DE
:1059800003501F4FFE01709690E0E80FF91F208131
:1059900030E0220F331F020F131FE02FF12F008181
:1059A000118100701C7F22E0829F20E0020E22E025
:1059B000121EF001E853F64F20813181202B312B4C
:1059C0002083318383958F3138F590E0FC01E35AD1
:1059D000F64F00810023B1F3FE01709690E0E80FCE
:1059E000F91F00810F3F09F086CFFE01E350FF4F02
:1059F000082F10E0000F111FE00FF11F008111812F
:105A000022E0829F20E0020E22E0121EF001E85305
:105A1000F64F00831183D6CF07E00E94BB1F80E0C2
:105A20008F3108F04FC1082F0E9445388395F8CF79
:105A300026E536E08E010E94631D0023C1F000E0E0
:105A40000E94E91F0E94F30E093519F0093709F089
:105A500039C10E94B1210E943622A0E0BA2F1A2F2C
:105A60000B2F0E940D2001E00093CC0C2BC121E5EF
:105A700036E08E010E94631D002341F42DE436E0E0
:105A80008E010E94631D002309F418C110E08824D0
:105A90002FEF3FE0A9010E94754B22EF3FE0A901E3
:105AA0000E94814B01E12FEF3FE0A9010E94814B51
:105AB00080E090E006C0FC01E853F64F0081100F33
:105AC0000196803002E09007B0F30091E709011BD6
:105AD0000A950093E7090EE20E94C20D80E090E073
:105AE0000BC0FC01E853F64F00819C012050384F59
:105AF000A9010E94814B0196803002E0900788F353
:105B00000091060C20E03AE0A9010E94814B00912F
:105B1000070C21E03AE0A9010E94814B80E090E06F
:105B200001C00196803002E0900770F49C01205083
:105B3000384FA9010E94754BFC01E853F64F1081C4
:105B4000011779F388248394EAECFCE00081118149
:105B500025EF3FE0A9010E94814B882009F075C024
:105B600025EF3FE0A9010E94754BEAECFCE02081A3
:105B70003181021709F069C00AEA24EF3FE0A90168
:105B80000E94814B08E001BD04EF11E00E94580C17
:105B900025EF3FE0A9010E94754B10E0EAECFCE024
:105BA00000831183EAECFCE0008111810F7F10700B
:105BB0000083118388240FEF24EF3FE0A9010E94A6
:105BC000814BEAECFCE00081118120E030E040E014
:105BD00052E060E070E00E94D44B2801390100E0FF
:105BE000400E00EE501E00E0601E00E0701E80E0DF
:105BF00090E001C00196803002E09007C0F49C0163
:105C00002050384FA9010E94754B602F8C0120E075
:105C100030E0040D151D261D371DF801322F3BBF46
:105C2000069000E00BBF601529F302E0802E20E013
:105C30003AE0A9010E94754B0093060C21E03AE07E
:105C4000A9010E94754B0093070C8820F9F40E946B
:105C500042210091DD09002361F0EAECFCE00081C3
:105C600011812091DD0930E020503F4FA9010E94B1
:105C7000814B00E115E10E9490490E943622A0E08C
:105C8000BA2F1A2F0B2F0E940D2009C005ED1DE021
:105C90000E94904900E3800E082D0E94C20D00E092
:105CA0000093CC0C22EF3FE0A9010E94754B2FEF2F
:105CB0003FE0A9010E94814BAD9804C008EE1DE0B1
:105CC0000E9490490091DC09091599F00091DC09C6
:105CD000013F20F000E00093DC0907C00091DC09DF
:105CE000083018F007E00093DC090E9456209090DD
:105CF000DC091A2F0B2F0E94EF210C94D8239A93C2
:105D00008A93802F082F0E942C4B0F3F2FEF1207F2
:105D100019F400E012E01CC0EAECFCE020813181C3
:105D2000232B51F090E0880F991FFC01E857F64FA4
:105D300020813181021B130B212F27FF03C000E0BC
:105D400010E006C0003024E0120710F00FEF13E05F
:105D50008991999108959A938A93902F812F02E0C7
:105D60000E94C20D0BE10E94C20D0BE50E94C20D04
:105D70008A3038F0082F4AE00E94854B005D0E946F
:105D8000C20D082F4AE00E94854B042F005D0E943F
:105D9000C20D0BE30E94C20D9A3038F0092F4AE081
:105DA0000E94854B005D0E94C20D092F4AE00E94AF
:105DB000854B042F005D0E94C20D06E60E94C20DB5
:105DC0008991999108959A938A93FA93EA933A92D2
:105DD0002A921A920A927A936A935A934A933A931E
:105DE0002A931A930A938FB79BB700E00BBF78945E
:105DF0000091CF0C002349F00091CE0C002321F03C
:105E000004E20E94C20D01C0D2D0E1EEFCE00081AC
:105E100011810F5F1F4F008311830091EE0D102F32
:105E200013951093EE0D0F70002309F06EC0E3EE92
:105E3000FCE000811181012B41F0E3EEFCE00081E8
:105E4000118101501040008311830091E00C002368
:105E500049F0E0EEFCE000810A95008308E015B30C
:105E6000102715BBAA9AA99A24B135B10091AF0D9C
:105E700010E003701070000F111FF801E955F24F88
:105E800020833183EFEAFDE00081039500830370F6
:105E900007B90091EF0D102F13951093EF0D0770B8
:105EA000002399F5EEE9FDE00081039500830E944F
:105EB000AF41879B2AC0969B28C00091DA0C002333
:105EC00021F500919A000F7700939A00959A969881
:105ED0000FE113E001501040E9F700C0000000910D
:105EE0009B00102F17FF0AC000919C00053531F46C
:105EF00004E110E00E94580C08E001BD969A9598C4
:105F000000919A00006800939A00E0EBFDE00081A8
:105F100007FF0CC00091EE0D002311F4A89815C0E6
:105F20000091EE0D083089F4A89A0FC00091EE0D93
:105F30001091B00D1023112341F40091B00D0023F6
:105F400021F001E015B3102715BB00E00093020D0E
:105F50009BBF8FBF0991199129913991499159910D
:105F6000699179910990199029903990E991F99165
:105F70008991999118959A938A93C80120E030E00D
:105F800010E20EEF0E944A4BECEDFCE0808391831F
:105F9000EEEDFCE08083918301E00093DB0C009345
:105FA000CF0C00E00093CD0C8991999108950E9447
:105FB000474C24970091DB0C002309F44DC000E00E
:105FC0000093311000E010E0E7E2F0E1008311837C
:105FD000E5E2F0E100831183E9E2F0E1008311835F
:105FE00000E00093980C03E000932F10CC2431C004
:105FF00002E0C09E800100501E4FF801E853F64FAA
:10600000208131810C2D10E0000F111FF801E450A8
:10601000F14F2083318300E010E02C2D30E0220F7F
:10602000331FF901EE53F04F008311832C2D30E024
:10603000220F331FF901EC50F24F008311832C2DF6
:1060400030E0220F331FF901E058F04F0083118335
:10605000C3940FE1C01660F2E5E2F0E10081118126
:10606000E7E2F0E1208131810217130708F05DC2F9
:10607000E5E2F0E1008111810F5F1F4F0083118382
:1060800000912F10033009F450C280E00CE190E041
:10609000FC01E857F84F0083839504E090E0FC0191
:1060A000E857F84F00838395CC246EC002E0C09E71
:1060B00000E0000E02E0101EF001E853F64F2081D0
:1060C0003181203004E0300768F00FEF13E022E068
:1060D000C29E20E0020E22E0121EF001E853F64FAD
:1060E0000083118390E0FC01E857F84FC08283954C
:1060F00001E010E02C2D30E0205E3F4FF901E75722
:10610000F34F408142954F700E94A34B90E0FC01F9
:10611000E857F84F0083839501E010E02C2D30E024
:10612000205E3F4FF901E757F34F40814F700E94C7
:10613000A34B90E0FC01E857F84F0083839502E001
:10614000C09E00E0000E02E0101EF001E853F64F82
:106150000081118190E0FC01E857F84F008383959E
:1061600002E0C09E00E0000E02E0101EF001E853C5
:10617000F64F00811181012F10E090E0FC01E857FB
:10618000F84F00838395C3940FE1C01608F0C8C18F
:10619000DD24F601E35AF64F00810023A1F30091BC
:1061A0002F10002309F092C00C2D10E0000F111FDA
:1061B000F801E25CF04F008111812C2D30E0220FBC
:1061C000331FF901E058F04F20813181021B130B7E
:1061D000212F220F220B322FE5E2F0E14081518185
:1061E00060E070E00E94D44BE7E2F0E14081518131
:1061F00060E070E00E941E4C2C2D30E0220F331F17
:10620000F901E058F04F40815181400F511F2C2D72
:1062100030E0220F331FF901EE53F04F40835183DA
:106220002C2D30E0220F331FF901E058F04F208170
:10623000318115950795020F131F212F220F220B75
:10624000322FE5E2F0E14081518160E070E00E9490
:10625000D44B40E950E060E070E00E94D44B4FE046
:1062600050E060E070E00E941E4C012F122F232F9F
:10627000330F330B2595179507952C2D30E0220F02
:10628000331FF901E858F14F008311830C2D10E002
:10629000000F111FF801E654F14F208131810C2DC0
:1062A00010E0000F111FF801E858F14F0081118133
:1062B000020F131F22E0C29E20E0020E22E0121EF7
:1062C000F001E853F64F0083118310C100912F10A5
:1062D000013009F046C00C2D10E0000F111FF8012D
:1062E000E654F14FA081B1810C2D10E0000F111F79
:1062F000F801EA5CF14F00811181212F220F220B5E
:10630000322FE5E2F0E14081518160E070E00E94CF
:10631000D44BE7E2F0E14081518160E070E00E94FF
:106320001E4C0A0F1B1F22E0C29E20E0020E22E03C
:10633000121EF001E853F64F008311830C2D10E07C
:10634000000F111FF801E25CF04F208131810C2D0C
:1063500010E0000F111FF801EE53F04F208331833E
:10636000C5C0DD24F601EC5FFF4E0081002309F07B
:1063700078C00C2D10E0000F111FF801E058F04F0D
:1063800000811181119501951040212F220F220BC0
:10639000322FE5E2F0E14081518160E070E00E943F
:1063A000D44BE7E2F0E14081518160E070E00E946F
:1063B0001E4C2C2D30E0220F331FF901E058F04F16
:1063C00040815181400F511F2C2D30E0220F331F8F
:1063D000F901EE53F04F408351832C2D30E0220F12
:1063E000331FF901E654F14FA081B1812C2D30E02B
:1063F000220F331FF901E058F04F208131811595AC
:106400000795020F131F212F220F220B322FE5E2D7
:10641000F0E14081518160E070E00E94D44B40E99E
:1064200050E060E070E00E94D44B4FE050E060E04C
:1064300070E00E941E4C012F122F232F330F330BBD
:106440002595179507950A0F1B1F22E0C29E20E095
:10645000020E22E0121EF001E853F64F0083118372
:1064600045C00C2D10E0000F111FF801E654F14F4C
:10647000A081B1810C2D10E0000F111FF801EA5C22
:10648000F14F00811181212F220F220B322FE5E2E3
:10649000F0E14081518160E070E00E94D44BE7E27E
:1064A000F0E14081518160E070E00E941E4C0A0FD3
:1064B0001B1F22E0C29E20E0020E22E0121EF0010D
:1064C000E853F64F008311830C2D10E0000F111FCD
:1064D000F801E25CF04F208131810C2D10E0000FBB
:1064E000111FF801EE53F04F2083318302E0C09E6C
:1064F00000E0000E02E0101EF001E853F64F0181AB
:1065000007FFD4CD00E010E022E0C29E20E0020EA2
:1065100022E0121EF001E853F64F00831183E2CD12
:10652000282F13E80EEF0E94F84700913110002346
:1065300021F000E00093CF0CA4C5E5E2F0E100817A
:106540001181E7E2F0E1208131810217130708F49D
:1065500098C500E010E0E5E2F0E100831183CC246F
:1065600027C002E0C09E00E0000E02E0101EF00115
:10657000E853F64F208131810C2D10E0000F111FE0
:10658000F801E654F14F208331830C2D10E0000F09
:10659000111FF801EE53F04F208131810C2D10E0D6
:1065A000000F111FF801E058F04F20833183C3948E
:1065B0000FE1C016B0F200912F10002309F09FC028
:1065C00001E000932F10EBE2F0E100811181EDE298
:1065D000F0E120813181220F331F021B130BE7E210
:1065E000F0E100831183CC2446C00C2D10E0000F95
:1065F000111FF801EC50F24F808191810C2D10E0B9
:10660000000F111FF801E858F14F00811181801B24
:10661000910B0C2D10E0000F111FF801E25CF04F00
:1066200000811181212F220F220B322FEDE2F0E1A8
:106630004081518160E070E00E94D44B4CE050E01A
:1066400060E070E00E94D44B45E050E060E070E014
:106650000E941E4C012F122F232F330F330B801B50
:10666000910B0C2D10E0000F111FF801EA5CF14FA7
:1066700080839183C3940FE1C01608F0D6C0DD2457
:10668000F601EC5FFF4E0081013009F0AECF0C2D1A
:1066900010E0000F111FF801EC50F24F0081118142
:1066A0002C2D30E0220F331FF901E858F14F2081E3
:1066B0003181021B130B212F220F220B322FE7E215
:1066C000F0E14081518160E070E00E94D44BEBE248
:1066D000F0E140815181EDE2F0E160817181461B82
:1066E000570B60E070E00E941E4C2C2D30E0220F12
:1066F000331FF901EA5CF14F00831183BBCF009196
:106700002F100130D1F502E000932F10EDE2F0E1FF
:1067100000811181E7E2F0E100831183CC240FE1D5
:10672000C01608F082C00C2D10E0000F111FF801F8
:10673000EC50F24F208131810C2D10E0000F111F21
:10674000F801EA5CF14F00811181201B310B0C2D07
:1067500010E0000F111FF801E858F14F008111817E
:10676000201B310B0C2D10E0000F111FF801EA5C0B
:10677000F14F20833183C394D2CF00912F10023088
:10678000B1F4E9E2F0E100811181012B61F003E055
:1067900000932F10E9E2F0E100811181E7E2F0E1DE
:1067A0000083118342C000E000932F103EC000918F
:1067B0002F100330D1F5CC2432C002E0C09E00E09F
:1067C000000E02E0101EF001E853F64F20813181E7
:1067D0000C2D10E0000F111FF801E450F14F208341
:1067E000318300E010E02C2D30E0220F331FF9013F
:1067F000EE53F04F008311832C2D30E0220F331F16
:10680000F901EC50F24F008311832C2D30E0220F60
:10681000331FF901E058F04F00831183C3940FE157
:10682000C01658F200E000932F1000912F100023A3
:1068300009F027C4E0E3F0E10081039500830091B3
:10684000301010919D0C011728F40091DB0C0023EF
:1068500009F4CBC00091DB0C0023F9F40091980CF3
:10686000002329F0E9E8FCE007850A9507870091F5
:10687000980C002391F40091CD0C002339F000E036
:1068800010E0ECEDFCE00083118307C00091A20C46
:1068900010E0ECEDFCE000831183ECEDFCE0008106
:1068A0001181012B21F401E0009331109EC000E022
:1068B0000093DB0CEAECFCE000811181ECEDFCE0E4
:1068C000208131810217130741F500E010E020E03C
:1068D00030E0E0EFFDE000831183228333830091F9
:1068E000980C002309F053C0ADE0B0E0A03400E004
:1068F000B00708F04CC0E0EFFDE00081118122817B
:1069000033810A0F1B1FF801E853F64F0081FD0188
:10691000E757F34F00831196E9CFECEDFCE00081DF
:10692000118120E030E0322F212F102F00E0110FD5
:10693000221F331F005010422F4F3F4FE0EFFDE06A
:1069400000831183228333830091980C0023F9F490
:10695000ADE0B0E018C0E0EFFDE040815181628120
:1069600073818D0120E030E0040F151F261F371FB3
:10697000F801322F3BBF069000E00BBFFD01E75747
:10698000F34F00821196A03400E0B00720F3E0EF4F
:10699000FDE00081118122813381005C1F4F2F4F68
:1069A0003F4F008311832283338300919D0C083075
:1069B00020F400919D0C002381F40BE01DE00E9467
:1069C0009049ECEDFCE0008111810E94C90E0DE5BB
:1069D0000E94C20D01E0009331100091980C002339
:1069E00009F43CCF00E000933010A0E0B0E020C0FC
:1069F000E0EFFDE00081118122813381A801B9011E
:106A00004F5F5F4F6F4F7F4FE0EFFDE0408351835B
:106A100062837383F801322F3BBF069000E00BBF07
:106A20008D01005C1D4FF801E853F64F008211966E
:106A3000A03400E0B00758F5EAECFCE000811181D9
:106A4000ECEDFCE0208131810217130789F6E0EFBD
:106A5000FDE00081118122813381F801E853F64F76
:106A600020818D01005C1D4FF801E853F64F208313
:106A7000E0EFFDE000811181228133810F5F1F4F24
:106A80002F4F3F4F0083118322833383D0CF009158
:106A900030100395ECEDFCE08081918110919D0C0C
:106AA000011708F44FC00091CD0C002339F000E02D
:106AB00010E0ECEDFCE0008311830BC00091980C1A
:106AC000023028F0ECEDFCE08081918102C08091E1
:106AD000A20C90E0EAECFCE00081118180179107A4
:106AE00059F400E410E020E030E0E0EFFDE0008346
:106AF00011832283338326C0882379F4E0EFFDE0FD
:106B000000811181228133810054104020403040A7
:106B1000008311832283338315C0082F10E020E007
:106B200030E0322F212F102F00E0110F221F331FD2
:106B3000005C1F412F4F3F4FE0EFFDE000831183CA
:106B400022833383A0E0B0E01BC0E0EFFDE0408192
:106B50005181628173818D0120E030E0040F151FA7
:106B6000261F371FF801322F3BBF069000E00BBFF6
:106B70008D0100581D4FF801E853F64F0082119621
:106B8000A03400E0B007D0F4EAECFCE00081118111
:106B90008017D9F6E0EFFDE0008111812281338179
:106BA0000A0F1B1FF801E853F64F20818D01005892
:106BB0001D4FF801E853F64F2083E1CF00913110CB
:106BC000002309F05EC20091460C10E045E00E94EF
:106BD000A34B40919F0C50E00E94AF4BE9E2F0E1E3
:106BE000008311830091470C10919F0C019F80013D
:106BF00045E00E94A94BD8010A2F0B2B11F4A1E00C
:106C0000B0E000E010E0CC240EC02C2D30E0220FCC
:106C1000331FF901EC50F24F208131810217130725
:106C200008F48901C3942FE1C21608F0E3C0DD2403
:106C3000F601E35AF64F20812223A1F32C2D30E0F8
:106C4000220F331FF901E450F14F4081518122E0BE
:106C5000C29E20E0020E22E0121EF001E853F64F21
:106C6000408351832C2D30E0220F331FF901E6546D
:106C7000F14F4083518320E030E04C2D50E0440F31
:106C8000551FFA01E858F14F2083318322E0C29E5C
:106C900020E4020E22E0121EF001E853F64F20819C
:106CA00031814C2D50E0440F551FFA01E857F64F43
:106CB00040815181240F351F432F47FF03C020E03F
:106CC00030E006C0203044E0340710F02FEF33E00E
:106CD0004C2D50E0440F551FFA01E450F14F408114
:106CE0005181B901641B750B4C2D50E0440F551FA9
:106CF000FA01EC50F24F608371834C2D50E0440F49
:106D0000551FFA01E450F14F608171814C2D50E024
:106D1000440F551FFA01E450F14F2083318342E0C4
:106D2000C49E40E8040E42E0141EF001E853F64F02
:106D3000008011804C2D50E0440F551FFA01E85798
:106D4000F64F40815181400D511D052E07FE03C0B5
:106D500040E050E006C04030E4E05E0710F04FEF46
:106D600053E06217730718F42417350730F026171D
:106D7000370728F44217530710F420E001C021E040
:106D8000222391F4E9E2F0E120813181232B61F4A7
:106D90002091301030E0E0919D0CF0E031972E17FB
:106DA0003F074CF0882339F420E0DD24F601EC5F46
:106DB000FF4E208306C021E0DD24F601EC5FFF4E8C
:106DC00020832C2D30E0220F331FF901EC50F24FBD
:106DD0004081518155230AF018CF2C2D30E0220F2D
:106DE000331FF901EC50F24F20813181319521950B
:106DF000304014CF48E250E00E94934BC8018D010F
:106E000043E050E00E94934BA8018C010E94AF4BDD
:106E1000EBE2F0E1008311830091A10C10E0EDE2C0
:106E2000F0E100831183EDE2F0E100811181000FB8
:106E3000111FEBE2F0E12081318102171307E8F125
:106E4000EAE5F9E0008102FF13C00BE50E94C20DE4
:106E5000009130100E94AB0D0CE20E94C20DEBE2DB
:106E6000F0E1008111810E94C90E0DE50E94C20D62
:106E7000EBE2F0E100811181012B39F400E010E038
:106E8000EDE2F0E10083118318C0EBE2F0E1008154
:106E900011810150104016950795EDE2F0E1008355
:106EA0001183EDE2F0E100811181012B31F400E06A
:106EB00010E0EBE2F0E100831183EBE2F0E100810E
:106EC000118120E030E0000F111F221F331FEDE27F
:106ED000F0E180819181A0E0B0E0880F991FAA1FA6
:106EE000BB1F081B190B2A0B3B0B48015901880CCF
:106EF000991CAA1CBB1C880E991EAA1EBB1E000F43
:106F0000111F221F331F088319832A833B83082DF7
:106F100009290A290B2929F49924AA24BB248824A5
:106F20008394088119812A813B81012B022B032B39
:106F300041F401E010E020E030E0088319832A8367
:106F40003B83CC2442C00419150926093709A40142
:106F5000B5010E941E4C2C2D30E0220F331FF90189
:106F6000E25CF04F008311830C2D10E0000F111F25
:106F7000F801E25CF04F20813181203004E03007DD
:106F80005CF00FEF13E02C2D30E0220F331FF901DE
:106F9000E25CF04F008311830C2D10E0000F111FF5
:106FA000F801E25CF04F2081318121300CEF300795
:106FB0005CF401E01CEF2C2D30E0220F331FF901AF
:106FC000E25CF04F00831183C3940FE1C01608F018
:106FD00050C00C2D10E0000F111FF801E058F04FC9
:106FE00000811181212F220F220B322FAC01BD0114
:106FF0000E94D44B280139010C2D10E0000F111F05
:10700000F801EC50F24F00811181212F220F220B49
:10701000322F0801190140E05AE060E070E0800181
:1070200091010E94D44B080119014CE050E060E04E
:1070300070E0800191010E941E4CDD24F601EC5F9E
:10704000FF4E4081442309F07ECF0419150926091B
:107050003709488159816A817B810E941E4C2C2D01
:1070600030E0220F331FF901E25CF04F00831183FF
:107070007BCFEDE2F0E100811181E7E2F0E10083F6
:1070800011832496EEE00C94584C0E944F4C402EF5
:107090005524F201E35AF64F0081002309F47EC023
:1070A00002E0409E800100501E4FF801E853F64F69
:1070B000018105FF06C020E018E1042D0E94424B2B
:1070C0006DC0EAECFCE000811181012BC9F002E007
:1070D000409E00E0000E02E0101EF001E853F64F63
:1070E000008111810F7F1370242D30E0220F331F98
:1070F000F901E857F64FA081B181A00FB11F0DC073
:1071000002E0409E00E0000E02E0101EF001E85395
:10711000F64FA081B181AF7FB3700B2F07FF03C083
:10712000A0E0B0E006C0A03004E0B00710F0AFEF80
:10713000B3E014E2042D0E942C4B0F3F23E0120712
:1071400058F4A017B10720F40A1B1B0BC80106C096
:10715000CD01801B910B02C008E010E09695879549
:1071600096958795883000E0900710F488E090E0CD
:107170000EE1009388070A2F00938907AB2FB0E038
:10718000A0938A07082F00938B07892F90E08093A4
:107190008C0725E013E0042D0E947348E6E00C9470
:1071A000604C0E94514CD8010091CF0C002309F093
:1071B00041C00A2F0B2BF1F1A03800E0B007D0F549
:1071C00000E010E0EAECFCE00083118380E00BC0FB
:1071D00022E0829F900120503E4FF901E853F64F84
:1071E0000083118383958F3110F590E0FC01E35A01
:1071F000F64F00810023B1F318E1082F0E941D4BC8
:10720000013029F41EE1082F0E947F2E04C014E2F1
:10721000082F0E947F2E003020E41207C9F60DEDE2
:107220001DE00E949049082F0E94AB0DDBCF8D011D
:107230000E94BB2FE4E00C94624C6AC00E94F30EE3
:107240001091E60C163018F010E01093E60C209127
:10725000E60C30E0F901E951F34F0083E6EEFCE083
:10726000108113951083053551F50091E60C0250FD
:10727000073008F00A5F10E0F801E951F34F008190
:107280000F3FE9F400E00093E60C0FEF2091E60CCD
:1072900030E0F901E951F34F0083E6EEFCE00081B4
:1072A0000395008305E52091E60C30E0F901E951F2
:1072B000F34F0083E6EEFCE000810395008300912C
:1072C000E60C063029F50091E70C0F3F09F5009117
:1072D000E80C0535E9F40091E90C1091EA0C1095E1
:1072E0000117B1F40091EB0C1091EC0C1095011703
:1072F00079F401E00093E50C3091EB0C20E0009173
:10730000E90C10E0020F131FE0EDFCE00083118395
:107310000091F00C1091EF0C011709F08FCF089538
:107320009A938A93C901083C09F0C8C0183119F42E
:107330008C0137DFFEC01A3111F01B3149F5E2ED47
:10734000FCE0808391830FEF0E94C20D05E50E944F
:10735000C20DE2EDFCE0008111810E94C20DE2ED60
:10736000FCE00081118100950E94C20DE2EDFCE07D
:1073700000811181012F10E00E94C20DE2EDFCE0BE
:1073800000811181012F10E000950E94C20DD1C033
:107390001F3159F4882311F401E001C000E0102FDF
:1073A00010FDAB9A10FFAB98C4C01232A1F540E0BB
:1073B00050E010E020E030E000E00E94AD0C00233F
:1073C00009F4B7C0E6EDFCE0008111810817190748
:1073D00039F040E050E010E09C0101E00E94AD0C6B
:1073E000EAE4F9E0038114810817190709F4A1C040
:1073F000EAE4F9E083839483082F23E030E0A901D5
:107400000E94814B892F90E0082F24E030E0A901F1
:107410000E94814B8EC0113229F4E3EEFCE08083A0
:10742000918387C0153221F48C010E94430E81C0E4
:10743000163251F48C010E94430E0DE00E94C20DE1
:107440000AE00E94C20D75C01832A1F540E050E07C
:1074500010E020E030E000E00E94AD0C002309F4D1
:1074600068C0E8EDFCE0008111810817190739F0C8
:10747000AC0110E020E030E004E00E94AD0CEAE452
:10748000F9E0018512850817190709F452C0EAE4EA
:10749000F9E081879287082F29E030E0A9010E9456
:1074A000814B892F90E0082F2AE030E0A9010E944B
:1074B000814B3FC002E010E8D1D43BC00436F0F06D
:1074C0000D36E0F42091CF0C222339F021E02093F7
:1074D000020D2091020D2223E1F7E4E3F7E1212FD1
:1074E00030E0E20FF31F2491223021F49C010E942E
:1074F0004A4B1FC0282F0E94424B1BC02091CF0C2B
:10750000222339F021E02093020D2091020D222345
:10751000E1F7ECEFF6E1212F30E0E20FF31F2491C9
:10752000223021F49C010E944A4B03C0282F0E9464
:10753000424B899199910895083C09F0E0C01831B7
:1075400029F4EEEDFCE0008111810895173229F451
:10755000ECEDFCE0008111810895193121F40091D6
:10756000CF0C10E008951A3111F01B3129F4E2ED2F
:10757000FCE00081118108951C3111F01D3149F4A6
:107580005CDE00E00093E50CE0EDFCE000811181A1
:1075900008951E3129F451DE0091E50C10E00895A4
:1075A0001F3141F405B306950695069500950170C7
:1075B00010E008951232B1F540E050E010E020E014
:1075C00030E000E00E94AD0C002339F1EAE4F9E07C
:1075D00003811481E6EDFCE020813181021713075D
:1075E000E1F0E6EDFCE000811181EAE4F9E00383DB
:1075F0001483E6EDFCE00081118123E030E0A90175
:107600000E94814BE6EDFCE000811181012F10E02A
:1076100024E030E0A9010E94814BEAE4F9E0038113
:1076200014810895143269F440E050E010E020E045
:1076300030E000E00E94AD0CE4EDFCE0008111813F
:1076400008951032B9F400E0809902C0006111E0A1
:107650000C9902C0086011E00D9902C0046011E0AD
:107660000E9902C0026011E00F9902C0016011E0A2
:1076700010E00895113229F4E3EEFCE0008111815D
:1076800008951832B1F540E050E010E020E030E01D
:1076900000E00E94AD0C002339F1EAE4F9E0018535
:1076A0001285E8EDFCE02081318102171307E1F03B
:1076B000E8EDFCE000811181EAE4F9E0018712873E
:1076C000E8EDFCE00081118129E030E0A9010E9491
:1076D000814BE8EDFCE000811181012F10E02AE0F0
:1076E00030E0A9010E94814BEAE4F9E001851285AE
:1076F000089501E010E8B2D30FEF1FEF08950436AC
:10770000E8F00E36D8F42091CF0C222339F021E096
:107710002093020D2091020D2223E1F7E4E3F7E12B
:10772000212F30E0E20FF31F2491223019F40E9440
:107730002C4B08950E941D4B10E008950F31D8F492
:107740002091CF0C222339F021E02093020D2091CB
:10775000020D2223E1F7ECEFF6E1212F30E0E20FFA
:10776000F31F2491223019F40E942C4B08950E949B
:107770001D4B10E0089500E010E008959A938A935D
:10778000E3E0FDE00081118198012F5F3F4FE3E0CE
:10779000FDE02083318320E030E0005010462F4F81
:1077A0003F4FF801322F3BBF0690002D10E01BBF6A
:1077B000E3E0FDE0408151819A012F5F3F4FE3E01C
:1077C000FDE02083318360E070E0405050466F4F11
:1077D0007F4FFA01362F3BBF0690202D10E01BBFD4
:1077E000E3E0FDE040815181CA010196E3E0FDE064
:1077F0008083918360E070E0405050466F4F7F4F30
:10780000FA01362F3BBF069010E01BBF002321F486
:10781000102D022F91DE4EC0023061F4102D30E0A9
:10782000220F331FF901E15FF24F20813181022FD6
:1078300083DE40C0013069F4002D10E0000F111FFD
:10784000F801E15FF24F00811181102F022F74DEE9
:1078500031C00330A9F4002D10E0000F111FF80112
:10786000E15FF24F00811181102F30E0220F331FB2
:10787000F901E15FF24F20813181022F5DDE1AC0F4
:10788000043039F4502D40E0022F10E0040F151F92
:1078900011C0053069F4102D00E030E0200F311FD9
:1078A000220F331FF901E15FF24F0081118102C005
:1078B00000E010E08991999108950E94514CA8012F
:1078C000E3E0FDE00081118198012F5F3F4FE3E08D
:1078D000FDE02083318320E030E0005010462F4F40
:1078E0003F4FF801322F3BBF0690002D10E01BBF29
:1078F000E3E0FDE000801180C0010196E3E0FDE0DF
:1079000080839183C001A0E0B0E080509046AF4FEB
:10791000BF4FFC013A2F3BBF0690602D10E01BBF0C
:10792000E3E0FDE000801180C0010196E3E0FDE0AE
:1079300080839183C001A0E0B0E080509046AF4FBB
:10794000BF4FFC013A2F3BBF069010E01BBF002346
:1079500029F49A01102D062FE3DC4BC0023069F4A4
:107960009A01102D70E0660F771FFB01E15FF24F67
:1079700040815181042FD4DC3CC0013071F49A0164
:10798000002D10E0000F111FF801E15FF24F0081A0
:107990001181102F062FC4DC2CC00330B1F49A01E2
:1079A000002D10E0000F111FF801E15FF24F008180
:1079B0001181102F70E0660F771FFB01E15FF24F1E
:1079C00040815181042FACDC14C0043021F407E065
:1079D00010E044D20EC0053061F4102D00E070E0DC
:1079E000600F711F660F771FFB01E15FF24F40834D
:1079F0005183E4E00C94624CC1DEE5E0FDE00083DD
:107A00001183E3E0FDE00081118198012F5F3F4F7A
:107A1000E3E0FDE02083318320E030E000501046B9
:107A20002F4F3F4FF801322F3BBF069000E00BBFB6
:107A300000920B0DA3DEE7E0FDE0008311830091CF
:107A40000B0D002379F4E5E0FDE000811181E7E012
:107A5000FDE0208131810217130711F401E0089540
:107A600000E0089500910B0D013079F4E7E0FDE0AE
:107A700000811181E5E0FDE02081318102171307CB
:107A800010F401E0089500E0089500910B0D02301C
:107A900079F4E5E0FDE000811181E7E0FDE020817F
:107AA00031810217130710F001E0089500E00895F6
:107AB00000910B0D033079F4E5E0FDE000811181C8
:107AC000E7E0FDE0208131810217130710F401E0A7
:107AD000089500E0089500910B0D043079F4E7E07B
:107AE000FDE000811181E5E0FDE020813181021798
:107AF000130710F001E0089500E0089500910B0DC8
:107B0000053079F4E5E0FDE000811181E7E0FDE07A
:107B1000208131810217130711F001E0089500E080
:107B2000089505E010E09AD100E0089500910C0D51
:107B3000013061F400910E0D002331F000910D0D24
:107B4000002311F001E0089500E0089500910C0D6C
:107B5000023061F400910E0D002321F400910D0D0F
:107B6000002311F001E0089500E0089506E010E020
:107B700075D100E008959A938A930230C9F0E3E04A
:107B8000FDE0408151819A012F5F3F4FE3E0FDE02E
:107B90002083318360E070E0405050466F4F7F4F4C
:107BA000FA01362F3BBF069010E01BBF00920A0D72
:107BB00010910A0D1F5F09F440C1125091F01A95FF
:107BC00009F11A9509F44CC01A9509F4F2C01A95F6
:107BD00009F4FBC01A9509F407C11A9509F41CC1F0
:107BE00037C1002331F0CADDE3E0FDE000831183FB
:107BF00032C1E3E0FDE0008111810D5F1F4F008382
:107C0000118329C1002319F1E3E0FDE00081118116
:107C10000D5F1F4F00831183B1DDE7E0FDE00083BE
:107C20001183E3E0FDE000811181065010400083E4
:107C30001183E7E0FDE0008111813FDEE3E0FDE03C
:107C4000008111810D5F1F4F0083118304C1E3E0A8
:107C5000FDE0008111810A5F1F4F00831183FBC08B
:107C6000002309F49DC0E3E0FDE0008111810D5F78
:107C70001F4F0083118382DDE5E0FDE00083118367
:107C8000E3E0FDE00081118198012F5F3F4FE3E0C9
:107C9000FDE02083318320E030E0005010462F4F7C
:107CA0003F4FF801322F3BBF069000E00BBF009220
:107CB0000B0D64DDE7E0FDE00083118300910B0D07
:107CC000002359F4E5E0FDE000811181E7E0FDE0EB
:107CD00080819181800F911F50C000910B0D013068
:107CE00059F4E5E0FDE080819181E7E0FDE000816D
:107CF0001181801B910B41C000910B0D023061F48A
:107D0000E5E0FDE000811181E7E0FDE04081518187
:107D10000E94934BC80131C000910B0D033061F4F8
:107D2000E5E0FDE000811181E7E0FDE04081518167
:107D30000E94AF4BC80121C000910B0D003159F4D6
:107D4000E5E0FDE000811181E7E0FDE080819181C7
:107D50008023912312C000910B0D013159F4E5E00D
:107D6000FDE000811181E7E0FDE080819181802BC1
:107D7000912B03C004E010E071D0E3E0FDE000814E
:107D800011810A501040008311838C0196DDE3E0DD
:107D9000FDE000811181095F1F4F008311835BC0EB
:107DA000E3E0FDE000811181065F1F4F0083118336
:107DB00052C0002309F04FC0E3E0FDE000811181D3
:107DC000E3E0FDE00083118346C0002321F00BE1D6
:107DD0000093090D40C0E3E0FDE000811181E3E084
:107DE000FDE00083118337C0002369F0E3E0FDE08C
:107DF000008111810D5F1F4F61D2C0DCE3E0FDE027
:107E00000083118328C0E3E0FDE0008111810D5F54
:107E10001F4F008311831FC0002331F079D2E3E0AC
:107E2000FDE00083118317C0E3E0FDE000811181D4
:107E3000E3E0FDE0008311830EC0002361F4E3E082
:107E4000FDE000811181E3E0FDE00083118303C0C8
:107E500003E110E003D08991999108959A938A9350
:107E6000C801EAE5F9E0008101FF1AC003E515E168
:107E70000E9490498C010E94C90E0BE50E94C20D20
:107E8000E3E0FDE0008111810E94C90E0AE30E9437
:107E9000C20D00910A0D0E94AB0D0DE50E94C20DAE
:107EA0008991999108950E94524CA02FAA2311F410
:107EB0009598969A00E010E0E3E0FDE000831183DE
:107EC00080E090E204E000930A0DAA2321F004E18F
:107ED00015E10E94904900E00093090D05C002E001
:107EE0004ADEAA2309F013D10091090D0B3109F4E0
:107EF00007C1E3E0FDE020813181203000EC300754
:107F000008F0FEC000910A0D053009F4F9C0E3E065
:107F1000FDE0008111810817190708F0F1C0E3E0C6
:107F2000FDE00081118198012F5F3F4FE3E0FDE00C
:107F30002083318320E030E0005010462F4F3F4F28
:107F4000F801322F3BBF069000E00BBF00920A0DF4
:107F5000EAE0FDE0008107FFC2CF00910A0D005862
:107F600049F00A9509F46FC00A9509F4B0C00A9562
:107F7000B1F1C2C041DD00930D0D00910D0D0093D4
:107F80000E0DE3E0FDE00081118198012F5F3F4F6E
:107F9000E3E0FDE02083318320E030E00050104634
:107FA0002F4F3F4FF801322F3BBF069000E00BBF31
:107FB00000920C0DAA2309F0AAD000910C0D002309
:107FC00009F092CF00910E0DD6DDAA2309F48CCFD3
:107FD00000910E0D002309F487CF99D085CF0CDDD9
:107FE00000930D0DA3DD00930E0DE3E0FDE0008195
:107FF000118198012F5F3F4FE3E0FDE02083318343
:1080000020E030E0005010462F4F3F4FF801322F54
:108010003BBF069000E00BBF00920C0DAA2309F0B5
:1080200076D000910C0D002309F05ECF00910E0D6B
:10803000A2DDAA2309F458CF00910E0D002309F404
:1080400053CF65D051CF00910E0D002359F0E3E0DE
:10805000FDE000811181085F1F4F0083118300E064
:108060008ADD42CFC9DC00930D0D00910D0D009308
:108070000E0DE3E0FDE00081118198012F5F3F4F7D
:10808000E3E0FDE02083318320E030E00050104643
:108090002F4F3F4FF801322F3BBF069000E00BBF40
:1080A00000920C0DAA2309F032D000910C0D002390
:1080B00009F01ACF00910E0D5EDDAA2309F414CF4A
:1080C00000910E0D002309F40FCF21D00DCFAA236C
:1080D00009F01DD000910E0D002311F401E001C044
:1080E00000E049DDAA2309F4FFCE00910E0D002324
:1080F00009F0FACE0CD0F8CE00E110E0AFDEF4CEFD
:108100000091CF0C0023E1F7E3E00C94634C0CE802
:1081100010E00E94904966D00DE20E94C20D0091CD
:108120000A0D0E94AB0D0AE30E94C20D00E20E94FC
:10813000C20D00910D0D0E94AB0D0DE30E94C20D0A
:1081400008E20E94C20DE5E0FDE0008111810E947D
:10815000C90E0CE20E94C20D00E20E94C20D009105
:108160000B0D0E94AB0D0CE20E94C20D00E20E94BA
:10817000C20DE7E0FDE0008111810E94C90E09E215
:108180000E94C20D00E20E94C20D00910C0D0E94DF
:10819000AB0D0BE70E94C20D00910E0D0E94AB0DBE
:1081A0000DE70E94C20D0BE50E94C20DE3E0FDE069
:1081B000008111810E94C90E0DE50E94C20D0E942E
:1081C000F30E0093090D0091090D0B3151F406E4F3
:1081D00015E10E949049E3E0FDE0008111810E94D9
:1081E000C90E089500910A0D003829F40DE515E136
:1081F0000E949049089500910A0D013829F405E67E
:1082000015E10E949049089500910A0D023829F461
:108210000DE615E10E949049089500910A0D03387A
:1082200029F405E715E10E949049089500910A0D8F
:10823000013029F40DE715E10E949049089500915D
:108240000A0D023029F405E815E10E9490490895CD
:1082500000910A0D033029F40DE815E10E949049C0
:10826000089500910A0D043029F405E915E10E94F2
:108270009049089500910A0D053029F40DE915E1A2
:108280000E949049089500910A0D063029F405EAEC
:1082900015E10E949049089500910A0D073029F4D4
:1082A0000DEA15E10E949049089500910A0D0F3FD3
:1082B00021F405EB15E10E949049089520919D0D50
:1082C0002A3010F520919D0D30E0220F331FF90167
:1082D000ED58F24F00831183EDE9FDE00081039535
:1082E000008320910E0D30E000919D0D10E0000FF5
:1082F000111FF801ED58F24F20833183EDE9FDE0C5
:10830000008103950083089509E010E0A7DD08953A
:1083100000919D0D0023E9F0EDE9FDE000810A9553
:10832000008310E0000F111FF801ED58F24F00819B
:10833000118100930E0DEDE9FDE000810A950083A7
:1083400010E0000F111FF801ED58F24F008111816C
:1083500008950AE010E082DD0FEF1FEF08950E94FC
:10836000514C00913210002309F0D3C00091510903
:10837000013009F094C0E7EAFDE002811381012B8E
:1083800009F45AC000E000939E0D00E010E0E3EA1B
:10839000FDE00083118300E010E0E3E3F0E10083FF
:1083A000118301E000933210E7EAFDE000811181C2
:1083B00045E050E00E94AF4B10E0EFE9FDE00083A4
:1083C0001183EFE9FDE080819181E7EAFDE0028120
:1083D000138145E050E00E94AF4B10E0801B910BF1
:1083E000E1EAFDE080839183E1EAFDE020813181D3
:1083F000243700E0300720F003E00093B00D1FC2E7
:10840000E1EAFDE020813181223700E0300720F0F1
:1084100007E00093B00D13C2E1EAFDE02081318155
:10842000203700E0300720F00FE00093B00D07C2C6
:108430000FE00093B00D03C200919E0D0370002366
:1084400009F0FDC1E7EAFDE00081118145E050E05F
:108450000E94AF4B10E0EFE9FDE000831183EFE9EC
:10846000FDE080819181E7EAFDE00281138145E032
:1084700050E00E94AF4B10E0801B910BE1EAFDE061
:1084800080839183E1EAFDE020813181293500E09C
:10849000300708F0D4C10FE70093B00DD0C1E7EA70
:1084A000FDE002811381012B09F0C9C100919E0DED
:1084B0000370002309F0C3C1E7EAFDE000811181E8
:1084C00045E050E00E94AF4B10E0EFE9FDE0008393
:1084D0001183EFE9FDE080819181E7EAFDE002810F
:1084E000138145E050E00E94AF4B10E0801B910BE0
:1084F000E1EAFDE080839183E1EAFDE020813181C2
:10850000293500E0300708F09AC10FE70093B00D5D
:1085100096C100913210013009F042C1E7EAFDE056
:1085200002811381012B61F400E010E01BBD0ABD44
:1085300000E00093B00DA89800E0009332107FC1D6
:1085400000919E0D0F71002329F400E010E01BBD87
:108550000ABD75C100919E0D0F71023009F06FC107
:10856000E7EAFDE00081118145E050E00E94AF4B59
:1085700010E0EFE9FDE000831183EFE9FDE0808189
:108580009181E7EAFDE00281138145E050E00E941D
:10859000AF4B10E0801B910BE1EAFDE080839183FB
:1085A000E3EAFDE000811181E1EAFDE02081318113
:1085B0000217130740F4E1EAFDE000811181E3EACC
:1085C000FDE000831183ECEFF5E1ABEABDE00D9136
:1085D0001C9111971695079516950795E00FF11FB9
:1085E000049110E0E5EAFDE000831183E1EAFDE09B
:1085F000008111810A5F1F4FEFE9FDE02081318189
:108600000217130718F00FEF13E010C00AEF17E17D
:10861000EFE9FDE040815181E1EAFDE02081318117
:10862000421B530B465050400E94AF4B003024E099
:10863000120710F00FEF13E01BBD0ABDA5EABDE065
:10864000ED91FC911197F69720F003E00093B00DA7
:1086500032C0A5EABDE0ED91FC911197F49720F0AE
:1086600007E00093B00D27C0E1EAFDE020813181F1
:10867000243700E0300720F003E00093B00D1BC06A
:10868000E1EAFDE020813181223700E0300720F06F
:1086900007E00093B00D0FC0E1EAFDE020813181D9
:1086A000203700E0300720F00FE00093B00D03C04A
:1086B0000FE00093B00DE3E3F0E1008111810F5F63
:1086C0001F4F00831183E3E3F0E1208131812836DD
:1086D00001E0300758F000E010E01BBD0ABD0FEFCD
:1086E0000093B00D02E800933210A9C0E1EAFDE06A
:1086F00020813181263700E0300758F000E010E09B
:108700001BBD0ABD0FEF0093B00D01E800933210BE
:1087100096C0E3EAFDE0008111810C531040E1EACC
:10872000FDE0208131810217130758F000E010E0CE
:108730001BBD0ABD0FEF0093B00D03E8009332108C
:108740007EC0E5EAFDE0208131812C3300E0300776
:1087500058F000E010E01BBD0ABD0FEF0093B00D14
:1087600004E8009332106BC0A5EABDE0ED91FC91E6
:108770001197F89708F463C0E1EAFDE020813181A8
:10878000203700E0300708F45AC000E010E01BBDBD
:108790000ABD0FEF0093B00D04E8009332104FC0F4
:1087A00000915109023041F002E00093510927E0A5
:1087B00030E0A9010E94814BE7EAFDE002811381CC
:1087C000012BC1F400E010E01BBD0ABD00E00093E6
:1087D000B00DA89800E000933210009151090023D9
:1087E00071F100E00093510927E030E0A9010E94F7
:1087F000814B25C000919E0D0F71002301F5E7EA22
:10880000FDE00081118145E050E00E94AF4B10E097
:10881000EFE9FDE000831183EFE9FDE080819181C4
:10882000E7EAFDE00281138145E050E00E94AF4B92
:1088300010E0801B910BE1EAFDE080839183E4E08E
:108840000C94624C07EE06B900E010E01BBD0ABDB7
:1088500003EC0FBD02E00EBD03E00093AF0DEFEAA5
:10886000FDE0008103950083037007B901E010E08B
:108870000E94580C24B135B10091AF0D10E0037087
:108880001070000F111FF801E955F24F208331835A
:10889000EFEAFDE0008103950083037007B901E072
:1088A00010E00E94580C24B135B10091AF0D10E0DA
:1088B00003701070000F111FF801E955F24F20836B
:1088C0003183EFEAFDE0008103950083037007B96F
:1088D00001E010E00E94580C24B135B10091AF0DB9
:1088E00010E003701070000F111FF801E955F24FEE
:1088F00020833183EFEAFDE000810395008303705C
:1089000007B901E010E00E94580C24B135B1009184
:10891000AF0D10E003701070000F111FF801E95542
:10892000F24F2083318308950E94524C1A981B9A6B
:108930000E94D40BA89800E00093580900935909AD
:1089400000E000935A0900935B0900E00093CF0C0C
:1089500000E00093E00C22E030E0A9010E94754B9A
:108960000F3FA9F021E030E0A9010E94754B0F3FB5
:1089700071F023EF3FE0A9010E94754B033038F4FA
:1089800027E030E0A9010E94754B033048F101E077
:1089900000934B0921E030E0A9010E94814B02E2E3
:1089A00000934A0920E030E0A9010E94814B00E0D9
:1089B00022E030E0A9010E94814B80E023EF3FE0FC
:1089C000082FA9010E94814B0AE00093E00C00E00F
:1089D0000093510927E030E0A9010E94814B37C084
:1089E00021E030E0A9010E94754B00934B0920E083
:1089F00030E0A9010E94754B00934A0923EF3FE044
:108A0000A9010E94754B802F23E030E0A9010E944C
:108A1000754B00934D0924E030E0A9010E94754B8D
:108A200000934E0929E030E0A9010E94754B0093A4
:108A300053092AE030E0A9010E94754B00935409C4
:108A400027E030E0A9010E94754B0093510900E036
:108A50000093520911E020E830E000E00E94B50BDD
:108A600021E010914A0900E00E94240C21E012E26A
:108A700001E00E94240C00E000935809009359097A
:108A8000E1DE789424EF3FE0A9010E94754B0535A3
:108A900019F400E060D45EC1833038F080E023EF49
:108AA0003FE0082FA9010E94814B94B700E004BF6A
:108AB00021EF3FE0A9010E94754B002361F0923045
:108AC00051F48395833008F080E023EF3FE0082FD6
:108AD000A9010E94814B9A70992361F40091510978
:108AE000002341F000E00093510927E030E0A901A4
:108AF0000E94814B21EF3FE0A9010E94754B01309C
:108B000031F001E021EF3FE0A9010E94814B00918B
:108B10005109023009F05DC000E8009332100FEFF8
:108B20000093B00D56C090E0809B04C002E310E0BB
:108B30000E94580C0091F00C1091EF0C011769F095
:108B40000E94F30EA02FA53521F40091EF0C0093A5
:108B5000F00C082F0E94C20D01C0A0E0882311F480
:108B6000AC9807C0813011F4AD9803C0823009F48D
:108B7000AE98933209F046C0A33209F043C004E135
:108B800010E00E94580C08E001BD809B04C002E385
:108B900010E00E94580C0C991CC002E310E00E94E7
:108BA000580C00915109002371F4E7EAFDE00281BD
:108BB0001381012B41F001E00093510927E030E0DF
:108BC000A9010E94814B0C9BFECF02E310E00E94A2
:108BD000580C809B31C0AD9AAC9AAE9A0091F00CC3
:108BE0001091EF0C011709F49ECF0E94F30E902F05
:108BF000953521F40091EF0C0093F00C082F0E94A2
:108C0000C20D92CF993011F0A93089F404E110E03F
:108C10000E94580C08E001BD8395833008F080E085
:108C200023EF3FE0082FA9010E94814BAECF9D307A
:108C300019F0AD3009F0A9CF21EF3FE0A9010E9462
:108C4000754B002331F000E021EF3FE0A9010E94C5
:108C5000814B809BFECF04E110E00E94580C00E99C
:108C600010E05ED326D3882391F401E074D3902FD3
:108C70000CE810E055D3092F0E94070F08E512E019
:108C80004FD301E000935A090E94170FFDCF0091C6
:108C90004A09013059F101E000934A0920914A093B
:108CA00014E00EEFEFD405E912E03AD300E814E83F
:108CB0002EE130E040914A0950E060E070E04F5F03
:108CC0005F4F6F4F7F4F0E941E4C0E94EA0D00EBDA
:108CD00012E026D300914A0920E030E0A9010E9469
:108CE000814B09B904EF11E00E94580C01E033D325
:108CF000902F0CE810E014D3092F0E94070F08E50D
:108D000012E00ED307E000935A0901E010E0EAEC0C
:108D1000FCE0008311830E944221E7EAFDE020810C
:108D20003181273302E0300730F023E333E012E2F1
:108D30000EEFB0D405C02FEF33E012E20EEFAAD44D
:108D4000813071F401E010E0EAECFCE00083118373
:108D50000E94362203E000935A090E94AA2312C0FF
:108D6000823081F402E000935A0900E00E94533FF0
:108D700004E610E00E94580C04E110E00E94580C38
:108D800008E001BDFFCFFA93EA934A933A932A93FE
:108D90001A930A933FB74BB700E00BBFAA982091F4
:108DA0009C000091EF0C10E00F701070F801EF5074
:108DB000F34F2083EFEEFCE00081039500834BBF6F
:108DC0003FBF09911991299139914991E991F991FF
:108DD0001895FA93EA934A933A932A931A930A932B
:108DE0003FB74BB700E00BBF00915809102F139508
:108DF000109358092CB110E0F801E857F94F20837F
:108E00004BBF3FBF09911991299139914991E9913E
:108E1000F9911895AA98A99808EA10E081D223C080
:108E20000E94F30E0E94BE0D5E9A0091F00C10910C
:108E3000EF0C0117A9F75E9BFECF1A981B9A0091C1
:108E4000590910915809011771F00091590910E062
:108E5000F801E857F94F0081E9E5F9E01081139531
:108E600010830E94C20D0091F00C1091EF0C0117BD
:108E700031F31B981A9AD9CF0E94504C902F44245A
:108E80009F3F29F400E91FE521E030E004C008EE2F
:108E900013E020E030E080E013C04091590950E039
:108EA000FA01E857F94F4081E9E5F9E0508153951F
:108EB0005083682F70E0FB01E65FF74F4083839596
:108EC0008917D8F440E050E060E070E00090590964
:108ED00010905809011479F40A011B01A001B10195
:108EE0004F5F5F4F6F4F7F4F001511052205330510
:108EF00068F744244394442081F2A82FB0E0009105
:108F0000C0080E3F09F470C0442071F09F3F61F02B
:108F1000EAE5F9E0008100FF03C00FE11DE000D2A7
:108F20000091580900935909A43008F45DC00091DC
:108F30000A080F3F21F400910B080F3F71F0EAE59A
:108F4000F9E0008100FF03C004E31DE0E9D10091D6
:108F500058090093590900E048C000910C0810918D
:108F6000C008011771F0EAE5F9E0008100FF03C0D5
:108F70000AE41DE0D5D1009158090093590900E099
:108F800034C020910D0830E00A2F10E0045010404A
:108F90002017310771F0EAE5F9E0008100FF03C016
:108FA00000E61DE0BDD1009158090093590900E089
:108FB0001CC082E007C090E0FC01E65FF74F008133
:108FC000B00F83958A17B8F3BF3F71F0EAE5F9E077
:108FD000008100FF03C006E71DE0A2D100915809FF
:108FE0000093590900E001C00A2FE5E00C94614CA0
:108FF0000E94514C3FEF3093BE083FEF3093BF08C3
:109000000093C008022F0E5F0093C1081093C2089E
:1090100080E00DC090E0FC01E857F84F0081A82FD8
:10902000B0E01596FD01E254F74F00838395821757
:1090300088F300E02A5FA22F82E007C090E0FC01E5
:10904000E254F74F1081010F839590E0EA2FF0E092
:1090500031978E179F0794F3009590E0FC01E2543E
:10906000F74F00831B981A9A80E009C05E9A90E03F
:10907000FC01E254F74F00810E94BE0D83958A17D0
:10908000A8F35E9BFECF1A981B9A0A2FE4E00C947B
:10909000624C0E94514CD801922F992359F40091AF
:1090A000C0080E3F21F400EF11E03AD103C001E106
:1090B00012E036D180E00CC0082F10E0FD01E00F77
:1090C000F11F00810E947A0E00E20E94C20D83957A
:1090D000891790F301E412E023D1092F0E94070FB2
:1090E000E4E00C94624C0E944F4C802F912F422E52
:1090F00001E00093CE0CB0E029C040E050E060E019
:1091000070E0F0E08A019B01A801B9014F5F5F4F59
:109110006F4F7F4F083EE3E01E07E0E02E07E0E0E0
:109120003E0778F40091590910915809011721F070
:1091300040E050E060E070E00F2FF02FF39505362F
:1091400008F30091580900935909B395B23008F01B
:109150004EC00091580900935909242D192F082F4A
:1091600047DFA02F913061F48E3F29F455245A94A3
:1091700050925C0930C006E0502E50925C092BC022
:10918000923039F45090890706E0500E50925C09F5
:1091900022C08E3FC1F08F3140F4082F10E0F8015B
:1091A000E35AF64F0081023870F0843680F08E3634
:1091B00070F4082F10E004561040F801E358F64F01
:1091C0000081023820F4552450925C0910C006E05A
:1091D000502E50925C09552009F4B7CF052D4CDE76
:1091E00000935C0900915C09051509F086CF00E049
:1091F0000093CE0C00915C09051509F443C0009161
:10920000C0080E3FF9F1EAE5F9E0008100FF15C062
:109210000DED1DE085D0082F0E94070F07EB10E031
:109220007FD02A2F0EEB18E034DF09EC10E078D065
:1092300020915C090AE018E02CDFEAE5F9E0008102
:1092400001FF1EC000E011E80E942E3F082F0E947F
:109250007A0E00E20E94C20D092F0E947A0E00E2EF
:109260000E94C20D009188070E947A0E00E20E94BF
:10927000C20D009189070E947A0E00E20E94C20D81
:1092800000E014C000915B09002379F007EB10E0C7
:1092900047D02A2F0EEB18E0FCDE09EC10E040D09E
:1092A00020915C090AE018E0F4DE01E0E6E00C94AD
:1092B000604C0BED10E034D000E814E82EE130E013
:1092C0004091990050E060E070E04F5F5F4F6F4F5A
:1092D0007F4F0E941E4C0E94EA0D00E20E94C20DC8
:1092E00000EB12E01DD00CE20E94C20D05EE10E072
:1092F00017D000E814E82EE130E049B150E060E01A
:1093000070E04F5F5F4F6F4F7F4F0E941E4C0E9477
:10931000EA0D00E20E94C20D00EB12E001D00895B8
:10932000EF97EF97A49720E001C02395203A60F4CF
:1093300030E0F801E20FF31F4491FE0130E0E20F4C
:10934000F31F4083442389F78E010E94E60EEF96B7
:10935000EF96A49608950E94514CB02FBB2361F064
:109360000CE810E0DDDF09E40E94C20D04E40E9475
:10937000C20D0AE30E94C20D90E020E011E00EEF62
:10938000B2DE00915C09002309F489C0A0E00EC0A0
:10939000843658F08E3648F420E0082F10E004564A
:1093A0001040F801E358F64F2083A39500915C0923
:1093B000A01708F074C00A2F10E0F801E65FF74F1D
:1093C00000810F3F91F70A2F10E00F5F1F4FF80148
:1093D000E65FF74F00810F3F41F70A2F10E00E5F65
:1093E0001F4FF801E65FF74F80810A2F10E00D5FF5
:1093F0001F4FF801E65FF74F0081023009F044C0CB
:109400000A2F10E00E5F1F4FF801E65FF74F408113
:1094100050E00A2F10E00D5F1F4FF801E65FF74F95
:10942000208130E0240F351F0A2F10E00B5F1F4F03
:10943000F801E65FF74F008110E0020F131F0F3FA6
:1094400020E0120709F58F3140F420E8082F10E0E2
:10945000F801E35AF64F20830DC0843658F08E365B
:1094600048F420E8082F10E004561040F801E358B3
:10947000F64F2083BB2331F0082F0E947A0E00E2C2
:109480000E94C20D939591CF8F3108F081CF20E0DB
:10949000082F10E0F801E35AF64F208386CF40EC06
:1094A00050EE60E070E080E059C002E0809F8001F3
:1094B000212F220F220B322F040F151F261F371FBB
:1094C0000F5F1F4F2F4F3F4FF801322F3BBF0690CA
:1094D000102D00E00BBF00E022E0829F212C220C27
:1094E0002208322C040E151E261E371EF001322DC6
:1094F0003BBF069020E02BBF1124000E111E082F49
:1095000010E0000F111FF801E857F64F008211829A
:10951000082F10E0000F111FF801E857F64F2081C7
:109520003181203000E4300769F0082F10E0000F8F
:10953000111FF801E857F64F20813181203000E4F7
:10954000300759F400E010E0282F30E0220F331FDD
:10955000F901E857F64F0083118383958F3108F4A2
:10956000A4CF80E010C014E2082F0E947F2E22E0DA
:10957000829F20E0020E22E0121EF001E853F64F17
:109580000083118383958F3180F5082F10E0F80157
:10959000E35AF64F00810023A9F310E1082F4DD0C4
:1095A0000068282F30E0F901E35AF64F008315E0F8
:1095B000082F43D0002321F020E015E0082F62D0CF
:1095C00018E1082F3AD0013071F61EE1082F0E94F1
:1095D0007F2E22E0829F20E0020E22E0121EF00188
:1095E000E853F64F00831183CDCF84E620C0A82F27
:1095F000B0E0A456B040FD01E358F64F00810023CF
:10960000A9F010E1082F19D00068A82FB0E0A456E7
:10961000B040FD01E358F64F008315E0082F0DD050
:10962000002321F020E015E0082F2CD083958E3602
:10963000F0F2092FE4E00C94624C1093880711E0DB
:109640001093890722E012E04EDD002319F000910B
:109650000F0808950FEF08951093880712E01093F4
:10966000890722E012E03FDD002349F03091100825
:1096700020E000910F0810E0020F131F08950FEF74
:109680001FEF0895109388072093890722E013E0C5
:109690002ADD089510938807122F10938907232F2E
:1096A00030E020938A0723E013E01DDD08950FE3E7
:1096B0000DBF05E00EBFC0E0D5E00E946D4C002359
:1096C00011F00E947F4C00E00BBF0E9494440E9466
:1096D000A24C0C94A24CE199FECF08954F5F5F4FCE
:1096E000FADF4EBB5FBBE09A0895FADF0DB3089531
:1096F0004F5F5F4F4EBB5FBBF894E29AE19A0FBE9B
:1097000008950FB6E8DF0DBBF5CF0024E8E0EA9539
:1097100032F0001F001C0416D0F3041AF8CF001F0B
:10972000402D00950895002411240030010741F0D8
:109730001695079510F4040E151E440F551FF5CF0E
:10974000002D112D08954A951AF0000F111FFBCF1F
:1097500008954A951AF016950795FBCF08950024B1
:109760001124EFE0001F111F001C111C0416150628
:1097700010F0041A150AEA95AAF7001F111F402DD0
:10978000512D0095109508953095209510950195CF
:109790001F4F2F4F3F4F08957095609550954195FD
:1097A0005F4F6F4F7F4F08950024112422243324EC
:1097B000E02FE12BE22BE32B71F0369527951795DF
:1097C000079520F4040E151E261E371E440F551F44
:1097D000661F771FEDCF002D112D222D332D0895FB
:1097E0004A952AF0000F111F221F331FF9CF089549
:1097F0000024112422243324E0E2EA9592F0001F91
:10980000111F221F331F001C111C221C331C0416A5
:1098100015062606370688F3041A150A260A370A9B
:10982000ECCF001F111F221F331F402D512D622D21
:10983000732D00951095209530950895FF27772377
:109840001AF4F1600E94CC4B33231AF4F0950E9475
:10985000C44B0E94F84BF69510F40E94C44BF69549
:1098600010F40C94CC4B0895AF93BF93B12FA02F5D
:109870003BBFD895EF5FFF4F3F4F0D924150504097
:10988000B9F74BBFBF91AF910895FA92EA92DA927D
:10989000CA92BA92AA929A928A927A926A925A92A8
:1098A0004A92BA93AA939A938A930895FF84EE8476
:1098B000DD84CC84BB84AA84998488847F806E8074
:1098C0005D804C80BB81AA8199818881F0E00FB6D0
:1098D000F894CE0FDF1F0FBE089501E0089520E039
:1098E00002D0E9F708952D9301501040202F212B2D
:1098F00008953BBF27913BB7F6DFD9F7089505E9F7
:1099000019E92801F20130E03BBF07911691F201FD
:109910003296A791B691F20134964791579166918C
:10992000242F252B262B21F0FA01362FE2DF01C050
:10993000D6DF07E0400E00E0501EA201433A59492D
:1099400008F3089500008895FECF141A1F24292ECD
:1099500033383D4D151B20252A2F343908080809B6
:109960000909090909090909090909090909090967
:109970000808080808080808080808070700FF037F
:10998000020504070609080B0A0D0C0F0E1110132F
:10999000121514160048014005A39900AD09880668
:1099A00000000049440050494E47004700474F001F
:1099B000445245534554005245534554005359535E
:1099C0005F57520041435400414354494F4E0052A7
:1099D00045475F5752005700575200575249544568
:1099E0000053594E435F5752005357520043414C66
:1099F0005500444543004845580043414C440052FB
:109A0000000D0A205B4349443A005D200052455452
:109A10000052455455524E0052554E0048454C5048
:109A2000005400544F535300434944005445535489
:109A30000043484B0044454D4F004D4F4E49544F55
:109A400052004241554400534541524348004C4561
:109A500044005343414E0055504441544500440096
:109A600044554D500042414C414E4345004F4646FF
:109A7000004F4E004E414D4500434F50590050009D
:109A8000504147450042004245464F5245004E0076
:109A90004E45585400474F544F004D4F4E005245CD
:109AA0000052440052454144004800455849540082
:109AB0005341560053415645004E4557004D004D09
:109AC0004952524F520053455400504C415900499D
:109AD00000494E534552540044454C455445004DB1
:0B9AE0004F5645005300535445500002
:00000001FF
